:10000000F01F001029570000275700002757000055
:100010002757000027570000275700000000000066
:100020000000000000000000000000002757000052
:10003000275700000000000027570000052500009A
:100040000D2300000D2300000D2300000D230000F0
:100050000D2300000D2300000D2300000D230000E0
:100060000D2300000D2300000D2300000D230000D0
:100070000D2300002557000025570000C100000097
:10008000A5250000BD250000D1270000E9270000BC
:10009000255700002D290000255700002557000096
:1000A0002557000025570000255700002557000060
:1000B0002557000025570000255700002557000050
:1000C000554B10B51A6801321A60544B1A68544BDC
:1000D000D2B2302A69D01ADC182A44D012DC082A9D
:1000E00032D0102A00D094E04E4A002111604E49CF
:1000F0000A68501C08604D49895C4D4AC9B21160BC
:10010000282287E0202A63D0282A32D081E0482A9A
:100110005ED004DC382A51D0402A53D079E0502AEE
:1001200060D0582A75D13F490A68501C0860404980
:1001300008684049C0B288543F4A0221FF3111602B
:1001400080221021D20563E0374A00211160116836
:10015000481C1060354A515C354AC9B211602822EA
:100160001A6001223CE030490A68501C08602F499F
:1001700009E02D4A314910680968884207D21168A0
:10018000481C1060294A515C294AC9B240E02C4AF7
:1001900011688022D205002901D0202138E02649AB
:1001A0000220FF300860102132E08022D2051021A9
:1001B000116008221A608122520011E08221490058
:1001C0001D4A25E01E4A1168042201291AD11DE0AA
:1001D0008022D2051021116008221A600422FF3209
:1001E000154B17E00F4A1168481C1060104804684E
:1001F0001048E4B244541068114A116804220139CD
:10020000884203D28021C9050A6002E01A6000E03A
:10021000116008221A6010BD98020010040000400E
:10022000180000408C02001094020010C00400105E
:1002300008000040B004001090020010D00400102C
:10024000AC0400101B4B02211A6810B50A431A6057
:10025000194B20211A68041C0A431A60174B1849CD
:100260001A680A401A601868012210431860154B7A
:1002700018680140196019680A431A60124B6C2211
:100280001A60124B1249186805F0D4FA114A10602E
:10029000114A1060022C02D1104BA0221A60104BA0
:1002A000802212021A6080234022DB0501201A609E
:1002B00010BDC046048004408080044030400440AB
:1002C000F8FCFFFF3440044018000040A404001074
:1002D000400D030014000040100000400C000040DE
:1002E00000E100E0034B1B689A06FBD5024B186047
:1002F0007047C0461480004000800040FFFFFFFFB1
:100300007FB5051C00200C1C01F0C4FA002801D0A8
:1003100002F0E2FE00262660281C2E60211C01F05F
:10032000E7FA301C01F0B6FAB04207D002F0D4FE72
:100330002660281C2E60211C01F0DAFA0C4B1B7879
:10034000002B13D00B4B2A6818680B49824203D14B
:1003500020680D68A84209D01A60236801A80B60C4
:10036000064902F015FD01A802F0BAFD7FBDC046A6
:100370009403001044010010480100105C59000073
:1003800038B5051C0C1C281C211C02F0B7F8024BC8
:100390001B68002BF7D138BD7002001008B502F0C1
:1003A000E1F808BD08B500230B60036001F0A0FA76
:1003B00008BD000010B502F057FE0D4B0020196873
:1003C00002F07CFA002002F069FA002002F046FAFE
:1003D000084B01241C60084B201C198802F02AF9E4
:1003E000201C02F017F9201C02F0F4F810BDC046E2
:1003F000A004001088020010A804001037B50C24D7
:100400000120032102F07AF8684601A9FFF778FF7E
:10041000009D002D02D1013C002CF1D1FFF7CAFF55
:10042000281C3EBD08B5002002F028FA012002F089
:10043000E1F802F01FFE08BD38B5051C0C1CFFF7E3
:10044000B9FF064AF823DB000121D150281C211CEA
:1004500004F08CFAFFF7E6FF38BDC046E004001058
:1004600010B5041CFFF7A6FF201C04F0B7F9041C0C
:10047000FFF7D8FF201C10BD08B50020FFF7F0FFE4
:1004800008BD000008B5021C0249034802F074FCD4
:1004900008BDC046725900006A590000F0B5314BE2
:1004A00085B01B68051C019304D0002B02D00020EE
:1004B00001F04EFC01F060F82B4C2C48236802211F
:1004C0000133032223602A4B01F044F92368013BE6
:1004D000236001F05BF8FFF7CFFF2648FFF7D2FF5C
:1004E000254F96239B003B6000243B689C4227DA03
:1004F00002F0FEFA002803D001F0C2FD002422E041
:10050000002D13D01D4EFA218900306805F092F9B4
:100510006423584302F00CF801F07CFEFA213068A5
:10052000890005F087F902F003F802E00A2002F0E2
:1005300019F802A803A9FFF7E3FE029B002B02D0E3
:10054000002D02D107E00134CFE7019B002B02D040
:10055000012001F0FDFBFFF78FFF094802F00CFCC2
:1005600005B0F0BD10000010040000107B59000021
:10057000BC6800008A59000090030010A404001019
:10058000905900001B4B73B5041C1B49186805F0FB
:1005900051F91A4900901A4A1A4B201C02F0F8FB34
:1005A00001F082FA002812D001F09AFAFA218900AB
:1005B000061C05F03FF9051C201C02F03AFC124B0A
:1005C00020186B431149F3182A1C02F0E1FB201C90
:1005D00002F02FFC0E4B20181B68002B02D003DA10
:1005E0000C4A02E00C4A00E00C4A0D4902F0D0FB34
:1005F00073BDC046A404001040420F00A159000082
:1006000072590000AE59000018FCFFFFB2590000FB
:10061000580100109E5900009B59000057690000C6
:10062000BD59000070B5051C0E1C141C00F0A4FF81
:10063000301C291C0022064B01F08CF8201C0121E3
:100640000922044B01F086F800F0A0FF70BDC046FF
:10065000BC680000A468000007B51449144A0120D2
:10066000FFF7E0FF642001F07DFF72B6114B00211F
:100670001960114B01221A6019601A601968012271
:100680001142FBD00D4B68461A600D4B8022196851
:1006900052020A431A600B4B80211A680A431A60FF
:1006A0003923009301A9084B984707BDC55900009D
:1006B00057690000708004407480044078800440D2
:1006C0008080044038820440F11FFF1F00B5084BB2
:1006D00089B01A78074B68461B78074902F058FB27
:1006E00001206946054AFFF79DFF09B000BDC046DD
:1006F0004C01001008000010F5590000035A0000DA
:10070000F0B52A4C2A4D237885B001932F78FFF756
:10071000DDFFFFF7B1FE002602A803A9FFF7F0FDF9
:10072000029800282BD0C0B201F032F840280CD03B
:1007300004D830280ED0392817D01BE0462830D0F6
:1007400049280DD0412815D126E02B783E2B11D811
:10075000013303E02B78002B0CD0013B2B7009E018
:100760002378062B06D8013303E02378002B01D031
:10077000013B237000F0ECFEFFF7A8FF0026029B70
:10078000002B02D0C82001F0EDFE04200321013629
:10079000FFF7F6FD1D2EBFDD019B2F70237000F0CB
:1007A000D7FEFFF769FE05B0F0BDC0460800001097
:1007B0004C01001038B5051C0C1C00F0A8FE291CCB
:1007C000221C0120FFF72EFF054B064A00219950FD
:1007D0001A1C94321168F522D200995038BDC046D7
:1007E000E0040010A407000010B590B06846FFF7C1
:1007F000C9FE00F0C1FE084C012168460A1C231CFA
:1008000000F0A8FF054801210922231C00F0A2FFE7
:1008100000F0BCFE10B010BDA4680000175A000024
:1008200000B52D228DB0002800D02B2268460D493E
:1008300002F0AEFA04A802F0E1FC0120694604AA25
:10084000FFF7F0FE03200021FFF79AFD0220FFF7DB
:1008500007FE0028EED00A200021FFF791FD0DB021
:1008600000BDC046505A0000F8B5041C161C0D1CF3
:10087000002702F0C3FC211C1431E774681C02F04D
:10088000E1FA00F079FE201C04213A1C0A4B00F02A
:1008900061FF0A4C281C04210922231C00F05AFF86
:1008A000BE4205D0064878210922231C00F052FFE1
:1008B00000F06CFEF8BDC046BC680000A4680000F3
:1008C0009069000010B58CB0FFF7D6FD124902A860
:1008D00002F0B8FA04A802A90022FFF7C5FF2E24EF
:1008E000FF34002204A802A9FFF7BEFF0020032165
:1008F00001F004FE0023684601A901930093FFF76D
:10090000FFFC009B002B02D1013C002CE9D1FFF73A
:10091000B3FD0CB010BDC046FDA80000F0B500242A
:1009200093B00594FFF7A8FD022296230194039249
:10093000271C5B00029300F01FFE019B9A4E002BC8
:100940006DD10AAD281C02F059FC019AEA742A7490
:100950006A73AA72EA712A71002C01D1012F05D1A4
:10096000281C04210022331C00F0F4FE8F4D331CA0
:10097000281C1E21002200F0EDFE8B4E012C01D11F
:10098000012F06D168462D3025210022331C00F0AE
:10099000E1FE281C33210022331C00F0DBFE824DD7
:1009A000022C09D1012F07D0684633304D21002297
:1009B0002B1C00F0CFFE09E00CA83A2100222B1CD2
:1009C00000F0C8FE032CEFD1012FEDD0784E2B1C88
:1009D000301C5921002200F0BDFE734D042C01D1C2
:1009E000012F06D1684636305F2100222B1C00F013
:1009F000B1FE301C6C2100222B1C00F0ABFE052C3C
:100A000001D1012F06D16846393072210022664B90
:100A100000F0A0FE0FA804210922664B03E06648FF
:100A200004210022331C00F095FE00F0AFFD059B71
:100A3000002B0AD0143B012B05D8052C03D096209F
:100A400001F090FD01E0FFF717FD0320011CFFF707
:100A500097FC002000F01EFF0023051C06A905A836
:100A600006930593FFF74CFC059B002B74D007AD54
:100A700008AE281C311C09AA02F0F4FB01900028E2
:100A800071D1281C02F0D8FC071C059812380528E3
:100A900068D804F06DFE0567240C6703601C00E055
:100AA000601D062104F01CFF00270C1C5BE0601E8B
:100AB000042804D804F05CFE060B0D103A002B88C5
:100AC000013316E0A8780C2104F0AAFE19E00137E2
:100AD0005FE0307801301BE07078013020E0601E6C
:100AE000042804D804F044FE0810121A22002B88AF
:100AF000013B2B80002445E0A8780C210A3004F04B
:100B0000EFFE0131A9703DE0013F42E0307817303F
:100B1000182104F0E5FE0422317040E070783B308B
:100B20003C2104F0DDFE0323717030E00023B3703C
:100B3000381C072104F0D4FE281C0A1C0991311C22
:100B4000052C02D102F0E9FB02E0039B02F0A4FBBA
:100B500001279623BB4008E0002D07D101235F4009
:100B60001F4003E0012796235B000293059B842B23
:100B700017D0182B15D0029B029A013B002A00D0F7
:100B8000D8E60EE0281C02F057FC0523071C03934F
:100B9000CEE7381C291C02F07FFC022405220392B8
:100BA000C6E713B0F0BDC046BC680000595A00004B
:100BB0004E5A0000A46800005B5A0000F7B502F02E
:100BC000B3FA18200021FFF737FC0024704DFFF71F
:100BD00029FC704EF8230022DB00F250201C02F0AA
:100BE000C4FA002C02D00020012101E006200321DC
:100BF00001F084FC201C02F0B3FA01A9071C68462E
:100C0000002F03D0FFF7CEFB012729E0FFF7CAFB37
:100C1000009A002A24D1002CE0D15F4B1B68002BE6
:100C2000DCD15C4B98331B68002B0BD15B4BED1870
:100C3000D4D500F055FC574B002294331A6002249F
:100C4000534DCBE7564B00941A6811321A60009A44
:100C5000102AEBDC03F0AAFD009B01330093F6E7BA
:100C6000002C0BD0009B182B01D0002FAFD000F030
:100C700095FC4C48FFF706FC0123F36600F042FFA9
:100C800002F0BCF9009A182A69D1019F0024F8B239
:100C900000F07EFDF823DB0001250194F5501928B2
:100CA00033D00FD8152835D007D811281ED01328D7
:100CB00052D1281CFFF7F2FB51E0162832D017283A
:100CC0003BD049E0262830D006D8212815D022284C
:100CD00042D104F0ADF942E0442836D045283BD15A
:100CE000E120000102F032FB281C32E02E4B1B6891
:100CF000002B34D0FFF7E6FD05E02B4B1B68002BE3
:100D00002DD0FFF70BFE009429E0284B1868281A15
:100D100001F01EF80120FFF767FDFFF7ADFBFFF7BD
:100D20006DFB1CE0FFF7ECFC19E0214B05221C7069
:100D3000204B1A7000F00CFC11E01F4B1A680132B6
:100D40001A60072A0BD11C6009E01C4802F0FEFA69
:100D5000201CFFF765FD02E000220197F250FFF72B
:100D600029FB0098019903F001FEF823DB00F358FA
:100D7000002B01D0FFF780FB064B94331B68002B40
:100D800003D100F0ADFB012420E704F06BFC1CE76D
:100D900020BF0200E0040010700200100CFEFFFFF4
:100DA0009C020010695A0000580100101000001049
:100DB0004C010010080000101C010010F0F1FFFFB2
:100DC00073B54B4D4B4B2A684B4C9A4202D12C6069
:100DD00001F05CF82B68A34202D1454B00221A6057
:100DE000464C02F06DF800F017FD4548002101F077
:100DF000DFF90021434801F0DBF900F0E5FD00F0E8
:100E000085FF23680726B3432360236801252B430E
:100E100000202360021C0B2101F054F9201C3A4CE5
:100E2000102101F0C5F923680022B3432360236831
:100E3000281C2360042101F045F9201C002101F049
:100E4000B7F901F029F99620000201F0ADFD2F4D10
:100E500001235B4200202B60FFF7C6FC00232B60C0
:100E600050240120FFF7EEF900F050FF02F026F9C0
:100E70002B68002B05D16420043C01F073FB142C7B
:100E8000EFD10020FFF7B0FC2821214802F06AFBD7
:100E9000142001F067FB1E48282102F063FB1D4867
:100EA00001F06AFF192001F05DFB01F021FE00282E
:100EB00003D00020FFF7F2FA02E0013C002CF1DC45
:100EC0001548082101F074F902F0AAFB03F00EFBAB
:100ED0001E2300930F23019310481149114A124B0E
:100EE00003F01EFB114803F04FFBFFF767FEC046FF
:100EF00008000010BE153E37E45BE1737440044007
:100F0000984004409C400440944004405801001024
:100F1000DE030000735A000010400440E156000058
:100F200001030000B50700009C02001088020010B9
:100F3000F7B500283BD00378303B5A425341C018E4
:100F40000378782B03D101301026012501E00A2611
:100F500000250378002201922D2B02D101230130BC
:100F6000019300230278002A1BD0171C303FFCB2EB
:100F7000092C02D87343DB1911E020273A43002DD6
:100F800008D0171C613FFFB2052F03D81B01573A49
:100F9000134304E0064801F0EFFE002007E00130B3
:100FA000E0E7019A002A00D05B420B600120FEBD01
:100FB0007D5A00000378202B01D10130FAE77047F9
:100FC000031C303BDAB2092A01D8181C0AE020239E
:100FD0001843031C613BDBB2052B01D8573801E0F5
:100FE00001204042704770B50E1CFFF7E3FF00255B
:100FF000041C2078002807D0FFF7E2FF002803DB5D
:101000002D0105430134F4E73560201C70BD00005C
:1010100008B500F065FD011C014801F0ADFE08BDFA
:101020008B5A000000B589B0684602F0E7F86946BF
:10103000024801F0A1FE09B000BDC046C75A000039
:10104000F7B50F1C01A9161CFFF772FF002814D07A
:10105000019C0B49201C04F043FC0D1C081C64215E
:1010600004F03EFC281C3970642104F0E3FB0449C1
:101070003070201C04F0DEFB01E001204042FEBD88
:101080001027000037B50D1C48686A4669460731CD
:101090000632FFF7D5FF01AC69466A46208001326F
:1010A000A8680231FFF7CCFF6B4618702288044B0A
:1010B0009A4203D9201C694602F02FF937BDC04679
:1010C0006B07000007B5486801A9FFF731FF019BD6
:1010D0003C20584302F03AF907BD0000072358436B
:1010E000054A10189C30013B04D3C25C002AFAD098
:1010F000002000E001207047E004001030B51948DE
:1011000085B001F039FE0024651CA30719D1201C0D
:10111000FFF7E4FF002810D0281CFFF7DFFF0028AE
:101120000BD0A01CFFF7DAFF002806D0E01CFFF769
:10113000D5FF002801D004340EE00B48211C01F03B
:101140001BFE211C684602F07FFA684601F0D2FEC1
:10115000064801F011FE2C1CFF2CD5DD01F0D8FE55
:1011600005B030BD72590000975A0000FCA800007D
:1011700070B50E1CFFF71EFF0D25041C0134631E05
:101180001878FFF71DFF002806DB7055013DF5D2EA
:10119000201CFFF70FFF00E0002070BD70B5444C2D
:1011A00086B023680868251C002B06D1414801F051
:1011B000E3FD03F09BF9012309E0012B0DD13E492A
:1011C000082201F048FE002803D123680133236080
:1011D0006BE03A4801F0D0FD5FE00378412B17D176
:1011E000374C0230211CFFF7C3FF002855D003788D
:1011F000422B52D1211C02300E31FFF7B9FF0028DB
:101200004BD00378432B48D1211C02301C3103E022
:10121000532B06D12B490230FFF7AAFF002844D1F7
:101220003BE04D2B1FD1284C0230211CFFF7A0FFC3
:10123000002832D003784E2B2FD1211C02300E31E2
:10124000FFF796FF002828D00378472B25D10230DE
:1012500001A9FFF7C8FE019B002B1EDB184A1B48A3
:1012600053651B491DE001A9FFF7BDFE047820234B
:10127000061C9C4311D1301C02A9FFF779FF019B8A
:10128000061CE118FF2902DC02A802F0F3F9002E87
:1012900003D00134042CEED107E003F027F90B480A
:1012A0000C4901F069FD00232B6006B070BDC046FB
:1012B0005C020010A05A000072590000B65A0000EB
:1012C000E0040010260500100A050010C25A0000B4
:1012D000DD590000CC5A000037B54C682378002B4C
:1012E00025D0201CFFF766FE01A9FFF77CFE019BBD
:1012F000041C002B1BD0D8B2FF2B09DD00F064FAD0
:10130000019B051C1812C0B200F05EFA019003E0C8
:1013100000F05AFA002501900198002802D0291CFB
:10132000FFF78AF823785A1E9341E418D6E737BDB1
:10133000064A08B5137801214B40137001D00449C7
:1013400000E00449044801F017FD08BD95030010B2
:10135000705A0000D35A0000D75A0000064A08B558
:10136000137801214B40137001D0044900E0044977
:10137000044801F001FD08BD94030010705A0000FC
:10138000D35A0000E65A000007B5486801A9FFF7E4
:10139000CFFD019B002B01DC01230193019B1E2B40
:1013A00001DD1E2301930199962292004A43034BCB
:1013B00003481A6001F0E0FC07BDC046900300102E
:1013C000F65A000008B50C4A1378013BDBB21370E3
:1013D000002B0AD0012B02D10849094A01E0094932
:1013E000094A0A4801F0C8FC04E0094801F0C4FCBD
:1013F000FFF732F908BDC046000000101A5B00007C
:10140000576900001E5B0000416C0000225B000079
:10141000465B000038B5051C002D09D0642402206D
:101420000021013C00F074FE002CF8D1013DF3E7EF
:1014300038BD70B5061C01200821021C00F092FE88
:10144000072401200821002200F08CFE321C012517
:1014500022412A400020022100F084FE281C08219D
:101460002A1C00F07FFE013CEBD270BD10B50021BC
:10147000041C0A1C022000F075FE201CFFF7D9FF97
:1014800010BDF0B5012385B002930023061C039321
:1014900072B6002402AB1B59502040421843C0B220
:1014A000FFF7E4FF0020FFF7E1FF1020FFF7DEFF6A
:1014B000E020FFF7DBFF212767430025F719022013
:1014C0000021012200F04EFE785D0135FFF7B1FFEB
:1014D000842DF4D10434082CDCD162B605B0F0BD03
:1014E00008B5AC20FFF7C2FFAE20FFF7BFFFA52075
:1014F000FFF7BCFF08BD38B50122051C0C1C00F02D
:10150000E1FD281C211C012200F02CFE38BD08B58D
:10151000AF20FFF7ABFFA420FFF7A8FF08BD08B579
:10152000AE20FFF7A3FF08BD10B5041CF820FFF79D
:101530009DFF201CFFF79AFF10BD10B5041C8120F1
:10154000FFF794FF3F202040FFF790FF10BD000001
:1015500008B5074B20201B781843FFF787FF0A20A8
:10156000FFF758FF034B1878FFF7E7FF08BDC046A9
:10157000080000104C01001008B584220248002128
:10158000520001F033FC08BD9603001008B5024874
:10159000FFF777FF08BDC0469603001008B501208D
:1015A0000821FFF7A8FF00200221FFF7A4FF022077
:1015B0000021FFF7A0FF02200621FFF79CFF032078
:1015C000011CFFF798FF0320011C002200F0CAFD58
:1015D00002200621002200F0C5FD06210122022082
:1015E00000F0C0FDFFF7C8FFFFF7D0FFA220FFF714
:1015F0003DFFA020FFF73AFFC020FFF737FF002094
:10160000FFF792FF0A20FFF705FF4020FFF72EFFAC
:101610002C20FFF72BFF3220FFF7FCFE2E20FFF7D8
:1016200025FF3220FFF7F6FE2F20FFF71FFF0A20CD
:10163000FFF7F0FEFFF78CFFFFF769FF08BD000022
:1016400083280ED80F290CD8CB08842253430722B5
:10165000C0181140034B80220A41111C1A5C11432F
:101660001954704796030010F7B55B18DBB201936D
:10167000019B994215D28425CC086C4307270F4063
:10168000802504193D41EFB2A618B44206DA054D93
:1016900065192B7801343B432B70F6E70131C9B251
:1016A000E6E7F7BD96030010F0B51E1C87B0059263
:1016B000F27804915B68824201D2307845E0244A96
:1016C000B478934205D10322041B54430192E418D9
:1016D0000CE0001B0022824204DA19780132023148
:1016E0005B18F8E71A789C1C5B780193A218002518
:1016F00003922F1C019B9F4226DA082200230292AC
:1017000000937378009A9A421CDA029A082A06D14A
:10171000039B9C4218D00022257802920134EB07EB
:1017200008D5049A009BB818059AC0B29918C9B296
:10173000FFF786FF009B029A013301326D10009380
:101740000292DEE70137D5E7019807B0F0BDC04649
:10175000615B0000F7B5041C0D1C161C1F1C01F07A
:1017600068FB20180190019B9C420DD0832D0BD863
:101770002078291C3B1C321CFFF796FF034B0134D9
:101780001B68C0182D18EEE7F7BDC0460400001016
:1017900010B50021012204230A4C0C5D844203D1C0
:1017A00018010243D0B20BE0013B002B04D10132FF
:1017B000092A00DD1A1C042301312829ECD100205C
:1017C00010BDC046CC6800000F23020918408000FD
:1017D000031F00D52833511E0020032906D8242BCF
:1017E00004DC04218A1A0249CB18985C7047C04671
:1017F000CC68000038B5051C0024054B291CE05CB2
:10180000044B0134C01800F0D3FC0A2CF5D138BDCC
:101810000869000000400440F8B50D4F3C68002CFA
:1018200015D11020FFF7E6FF0A4B0022E65C1B19DA
:101830005D78301C291C00F045FC0234301C291C4A
:10184000012200F08FFC142CEED101233B60F8BD87
:1018500050010010F468000070B500240B4B012209
:10186000E65C1B195D78301C291C00F02BFC02344F
:10187000301C291C002200F075FC142CEED1002035
:10188000FFF7B8FF024B00221A6070BDF468000039
:101890005001001038B5051CFFF7BEFF002D09D020
:1018A00007210122022000F00DFC104B80211A6854
:1018B0008A431A6000200B2100F02AFC0124002832
:1018C00005D000200B2100F023FC44424441002DB0
:1018D00009D007210022022000F0F4FB034B8021F5
:1018E0001A680A431A60201C38BDC046FC3F0250EB
:1018F000F0B587B00026029001200391049605966A
:10190000FFF7C8FFB04202D018230493012600213C
:10191000284C009120786178012200F0D3FB2078D8
:101920006178002200F01EFC234B9D1D012E24DC5B
:101930006A782F78111C381C019200F0E9FB00280E
:1019400008D100991D4AB3008A5C103369465A5089
:1019500001360BE02878697800F0DAFB0028F0D037
:10196000381C019900F0D4FB0028EAD0009A144BEF
:101970000132023D00929D42D8D127786578381C0B
:10198000291C002200F09EFB291C381C012200F0BB
:10199000E9FB0C4902348C42BCD10020864206D0BF
:1019A000049A029B05991A60039A0120116007B0FE
:1019B000F0BDC046F4680000C4680000CC680000B8
:1019C000C26800000869000008B50120021C0B2154
:1019D00000F078FB01200B21002200F0C3FB032064
:1019E0000221012200F06EFB03200221002200F000
:1019F000B9FB08BD234B37B51A6810218A431A601A
:101A0000214B8022196892010A431A60051C0B21A0
:101A10000120002200F056FB01200B21002200F0E3
:101A2000A1FB1A4B9F211A68194C8A431A601A6845
:101A300018491A60184B186803F0FCFE8023000256
:101A400018432A1C20600221032000F08BFB142085
:101A500000F088FD2368FF229343236023680F4A28
:101A6000134323600E4B1B680193019B002BF9DA93
:101A700022680C4B13402360FFF7A6FF0198000477
:101A8000800D3EBD38820440808004409840044070
:101A900000C0014000093D00A404001080000001C6
:101AA0002CC00140FFFFFFF810B50C4C2068002847
:101AB00013DA00202060FFF79DFF0A280ADC0120CE
:101AC000FFF798FF0138C023FF385B00984201D828
:101AD00001232360FFF778FF206810BD0C00001081
:101AE00008B5FFF7E1FF002801D1002007E0012041
:101AF000FFF780FF011EF8D0014803F09BFE08BDF0
:101B000050BB120008B5FFF7CFFF00280AD0FFF73F
:101B1000E7FFFA22031C0021C00FD2009A4248417D
:101B2000014B186008BDC0465401001008B5074BB2
:101B300002221A60064BA2221960064B1A70A322D9
:101B400058709A7000F00AFE08BDC046D00400101C
:101B5000AC040010C004001008B5064B0231196037
:101B6000054B00221A60054BA2221A70587000F033
:101B7000F5FD08BDD0040010AC040010C004001036
:101B800070B5051C0E1C0324281C311CFFF7CEFF6A
:101B90000223FF33984202D0013C002CF4D170BDE7
:101BA00070B5051C0E1C0324281C311CFFF7D4FF44
:101BB0000223FF33984202D0013C002CF4D170BDC7
:101BC0000B4B10B51C6800239C420ED0094CA31C83
:101BD000A270140A5C70140C120EDA709C70FFF77D
:101BE000DFFF831EFF3B5A425341181C10BDC04605
:101BF00058010010C004001070B50E4C2568002478
:101C0000A54215D00C4C160AA270E670160C120EE6
:101C10006271A371A21D26711C0A54701C0C1B0E4C
:101C20009470D370FFF7BCFF841EFF3C63425C419D
:101C3000201C70BD58010010C004001008B5064BF0
:101C40001A6800239A4205D0FFF79AFF831EFF3BD4
:101C50005A425341181C08BD5801001008B5074BE3
:101C600000201B68834207D002200721FFF788FF6E
:101C70000238FF384342584108BDC04658010010A1
:101C800038B50F4B051C1B680020834217D0092470
:101C9000641B631E062B10D8072C05D00948A91E0B
:101CA0000918221C01F080F8E8B2211CFFF778FF28
:101CB0000238FF384342584101E00120404238BD1C
:101CC00058010010C2040010012010B5011CFFF7DC
:101CD00057FF0223FF3398420ED1094B01211960AF
:101CE000084B1C78230709D0074B032222409A7027
:101CF000081CFFF755FF01E001246442201C10BDC1
:101D000058010010B0040010C004001008B5FFF71F
:101D1000DBFF02200121FFF733FF0223FF3398424C
:101D20000FD1084B1B787F2B06D984220220072174
:101D30005204054BFFF760FF09200421034AFFF717
:101D40003FFF08BDB00400100201140080808080B5
:101D500010B500280CD0254B80211A688A431A60E0
:101D6000234B1B68D907FBD5224B03221A6001E0E5
:101D7000204B1860204B012200211A6019601A6064
:101D8000196801221142FBD01C4B80211A601C4AA9
:101D900049021468214311601A1C002804D1134B16
:101DA0008024196821431960164B196888421CD099
:101DB0001860002801D0144800E01448116803F0AE
:101DC000EBFC134BFA2118608900041C03F032FD70
:101DD0001E2358430F4BC82118604901201C03F0F3
:101DE00029FD0D4B186001F055F810BD38820440F4
:101DF0000C8004407080044074800440788004406B
:101E00008080044010000010006CDC02001BB70052
:101E1000A4040010A0040010A804001008B500F0ED
:101E200043F9134B00211A68120B12031A60114B6D
:101E30001A68120B12031A600F4B1A68120B120366
:101E40001A600E4B1A68120B12031A600C4B012217
:101E500019600C4B1A6019601A601A68D107FCD51A
:101E6000094B23221A600020FFF772FF08BDC0460D
:101E7000008000500080015000800250008003501C
:101E8000408004404480044008800440014A024BE2
:101E90001A60FEE70400FA050CED00E038B50C49C5
:101EA0000C4800F069FF0C4D0024281C00F064FF72
:101EB0000A4A0B48A1581219D2682B1C143400F09E
:101EC0005BFFF02CF4D1074800F056FF38BDC04648
:101ED0007259000012690000556900009C6A0000F8
:101EE000246900002F690000F0B5404B8BB01E68DC
:101EF000041C002E01D1351C0AE03D4B02901B68EA
:101F000001209B6802A998475EE033681E79019D15
:101F10002378002B31D0082D33D02378202B01D10A
:101F20000134FAE7002B28D06A1CAD0008356B4657
:101F30000192EC50FF2E54D02278002A07D0631C67
:101F4000202A01D01C1CF7E7002222701C1C019AD9
:101F5000012ADCD1264E274B0D253360371C013D6D
:101F6000002D36D03B680298196800F085FF0028E4
:101F7000CBD03B6814333B60F1E7002D24D0022D19
:101F800002D0B54206D911E003981B4900F074FF56
:101F90000028F6D1164C19482368D96800F0ECFEE9
:101FA00023681748196900F0E7FE0DE0104CE8B20D
:101FB000236802A99B68984723689A68114B9A4244
:101FC00002D0114B03221A70084A1368002B0BD160
:101FD00003E0281C291CFFF761FF0C4800F0CCFE31
:101FE00002E0019D0026CAE70BB0F0BD5C020010C4
:101FF000640200109C6A00009F59000051690000B3
:10200000C75A0000C5130000000000105869000006
:1020100038B5041C164D0A2808D002D8082811D05B
:102020001CE00D2802D07F280CD017E02A6800237E
:102030001370104800F0A0FE0F4C201CFFF754FF57
:102040002C6013E00C4B2A689A420FD90B48211CD4
:1020500000F092FE2B68013B2B6007E00748211C33
:1020600000F08AFE2B685A1C2A601C7038BDC046DE
:1020700060020010556900005C01001064690000F6
:1020800008B500F035FD002804D000F007FDFFF78B
:10209000BFFFF6E708BD0000014A024B1A60704717
:1020A0005C01001060020010044B40211A680A43D2
:1020B0001A60034B01221A707047C04680800440AA
:1020C000680200100F4B70B51B78061C0C1C151C09
:1020D000002B01D1FFF7E8FF701E022803D80A4B3E
:1020E0008000C35800E0094B1A68012D04D1A540B7
:1020F0002C1C14431C6003E00121A1408A431A6098
:1021000070BDC046680200108C6B0000008000505B
:1021100038B50F4B051C1B780C1C002B01D1FFF7A9
:10212000C3FF0020032D12D8281C012203F020FB3E
:1021300002040608074B04E0074B02E0074B00E0EF
:10214000074B1B68A2401340181C421E904138BD2B
:1021500068020010FC3F0050FC3F0150FC3F025061
:10216000FC3F03500F4B70B51B78061C0C1C151C54
:10217000002B01D1FFF798FF701E022803D80A4BED
:102180008000C35800E0094B1A68012D04D1A54016
:102190002C1C14431C6003E00121A1408A431A60F7
:1021A00070BDC04668020010986B0000FC3F0050F4
:1021B00038B5084B041C1B780D1C002B01D1FFF710
:1021C00073FF236818229343236023681D4325600F
:1021D00038BDC04668020010054B3F221A60054B0F
:1021E00001221A60044B40211A688A431A60704722
:1021F00024800440D88004403882044008B5044B51
:1022000040211A688A431A60FFF7E6FF08BDC046FE
:1022100038820440094B0A4A19680A408021490063
:102220000A431A60074B04211A688A431A60064B56
:102230001A68064B1A6030BF7047C04600800340E2
:10224000FFF7FFFF10ED00E03882044034820440C5
:1022500008B500F049FAFFF7FFFA0A480021FFF736
:10226000A7FF09480021FFF7A3FF08480021FFF757
:102270009FFF07480021FFF79BFF06480021FFF75B
:1022800097FF08BD0840044000400440AC400440B3
:10229000144004401C40044008B50120FDF7D2FF63
:1022A00008BD000008B5124B8022DA675200DA67D9
:1022B0008022D200DA6780225201DA67802212017E
:1022C000DA6780229200DA670A4A0023136001214C
:1022D000094A49421160094A1360094A1360094AD0
:1022E00001231360084A1360FFF7D6FF08BDC046FC
:1022F00004E100E0048204400882044004C000407D
:102300003CC0004000C000400040014008B5064B02
:102310001A6801321A60054B1868FFF719FDFFF7BC
:10232000C1FFC046C04608BD6C020010100000107E
:10233000F7B5071C0C1C72B6FFF78AFF524B1A68E0
:10234000524B1A60002F01D0514B00E0514B524AC2
:1023500004211360514B524D1A680A431A6000233E
:102360002B60A1071ED04F4B4F4A19680A401A60D4
:1023700029684E4BA2070ED5EC2252010A432A606F
:1023800080221A6052001A608022D2001A608022D5
:1023900052011A6003E0802212010A432A6080225F
:1023A00012011A60002F53D0414B00241C60414B96
:1023B000414E1C60414B301C1C60414B211C1C6079
:1023C000FFF7F6FE201C0921221CFFF77BFE201CD4
:1023D0000921221CFFF7C6FE3A4B80211A683A48B1
:1023E0000A431A603368072293433360336802223A
:1023F000134333600A21784303F0CEF9334B0322B1
:102400001860334B1C60334B1A60334B334A1968E6
:102410000A401A601A6880210A431A60234A8B0016
:102420001360204A1168194311602A68022113437E
:102430002B602B4B01221A602A4B19602A4B1C4936
:102440001A601C601A60186801221042FBD00A60F2
:10245000264B012252421A60254B00221B68019331
:10246000244B1A6062B630BFC046214B019A1B68EC
:102470009A4208D11F4B01221A601F4B1868FFF7C0
:1024800067FCFFF70FFFF7BD388204403482044039
:10249000BF180000FF1800003082044010ED00E07B
:1024A00004820440008204407FE2FFFF00E100E07C
:1024B00004C0004004000140644004400440014066
:1024C0000480014080800440841E000018C0004049
:1024D00008C0004014C000403CC000400FF0FFFFA7
:1024E0007880044070800440748004400882044076
:1024F0006C020010700200101000001008B5FFF709
:1025000017FF08BD074B1A68013203D1064A11684C
:10251000013111601A6801321A60044B1A680132E5
:102520001A607047800200107C02001074020010D4
:10253000074B98420AD8074A00231360064A01381D
:102540001060064A1360064B07221A607047C046A7
:10255000FFFFFF008002001014E000E018E000E040
:1025600010E000E00B4A10B51368002800D10120EC
:10257000C1438B4208D91168994209D3591C146888
:1025800009188C42FAD3F6E71168C91A8142FBD3C5
:1025900010BDC04680020010014B18687047C0464D
:1025A00080020010034B01221A60034B1A680132AB
:1025B0001A60704700C0004084020010034B0122E3
:1025C0001A60034B1A6801321A607047000001401C
:1025D00088020010002803D1044B01221A6003E096
:1025E000012801D1024B18607047C04604C000406A
:1025F00004000140002802D1044B186004E00128C7
:1026000002D1034B00221A607047C04604C000404C
:1026100004000140002801D1044B02E0012804D14C
:10262000034B1A6802210A431A60704704C0004035
:102630000400014010B5002900D1134900280DD134
:10264000124B80241A6822431A60114B032218602F
:10265000104B1960104B1A60620211E0012811D171
:102660000A4B80221868520002431A600B4B00226A
:102670001A600B4B032219600A4B1A6080229202E7
:10268000094B1A6010BDC046FFFF00008080044067
:102690008402001018C0004014C0004088020010DE
:1026A000180001401400014000E100E080231022E6
:1026B000DB051A60094B08221A6000238022D2052C
:1026C0001268D10604D5064A934201D00133F5E7DA
:1026D000044898429B4158427047C0461800004049
:1026E000FF0F0000FE0F000008B58022154B1202FC
:1026F000DA67154B6C221A60144B154A19680020D2
:102700001140196019681960124B19680A401A6063
:102710001A6804211A600122FFF7D4FC002004216A
:102720000122FFF71FFD002005210122FFF7CAFC4F
:10273000012200200521FFF715FD074B00221A603A
:1027400008BDC04604E100E01800004030400440ED
:10275000F8FCFFFF3440044004800440F8B5174AF9
:10276000174C002323601360164A20211360802237
:10277000D20511602168144A012903D0934203D085
:102780000133F7E7934203D1FFF790FF002014E0F5
:102790000E4F00253E68013E2368FF2B0CD83B6896
:1027A0009E4204D03E68FFF7F7FE051C0A35FFF78E
:1027B000F3FE8542F0D1E7E72068F8BD8C020010F7
:1027C0009002001094020010FF0F00009802001009
:1027D000034B01221A60034B1A6801321A607047DA
:1027E000004001409C020010174B70B501241C6092
:1027F000164B1A6812191A60154B1A68002A22D053
:102800001A68144D013A1A601E68002E0DD02A680D
:10281000201C211CFFF7A6FC2B68201CE31A2B6050
:102820002A680221FFF79EFC0DE01B68201C2B602C
:102830002A68211CFFF796FC2A68201C0221FFF75A
:1028400091FC054B1E6070BD00800140A402001089
:10285000A0020010A802001004800140002803D14B
:10286000044B01221A6003E0012801D1024B1860D9
:102870007047C0460440014004800140002802D156
:10288000044B186004E0012802D1034B00221A60B7
:102890007047C0460440014004800140002801D137
:1028A000044B02E0012804D1034B1A6802210A43B9
:1028B0001A607047044001400480014010B50028B0
:1028C0000FD1124B80221C68920022431A60104BD9
:1028D000032218600F4B19600F4B1A608022D2023E
:1028E00011E0012811D1094B80221868D20002435F
:1028F0001A600A4B00221A60094B03221960094B27
:102900001A6080221203084B1A6010BD80800440B8
:102910009C0200101840014014400140A402001025
:10292000188001401480014000E100E008B5184B18
:102930001A680E231340062B0DD1164B9E221B68DE
:10294000134205D0144ADBB25360144B1B681EE0DF
:10295000D9071CD501E0042B05D1104B1868C0B273
:1029600000F0B1F813E00C2B06D10B4B8022596814
:1029700052000A435A600AE0022B08D1054B1A683C
:10298000054B910601D5002200E001229A6008BDA6
:102990000880004014800040AC020010008000401D
:1029A00000487047AC020010F7B52D4B2D4C80222B
:1029B000002192030191061CDA67201C902200F08E
:1029C00015FA019B0725A360274B284F1A68AA43D5
:1029D0001A601968012211431960254B1968A9432F
:1029E0001960196811431960224B80211868490148
:1029F00001431960204B1A6083223A601F4A126813
:102A000019681F4B1868504302F0C6FE311C0009BC
:102A100002F0C2FE1B4B10221B491A60030A0B6016
:102A20001A4BC0B2032218603A60194A1560194A5D
:102A30001D1C10680190106860230340602BFAD1C0
:102A400010680123184202D02B680193F8E7237025
:102A50008022114B92031A6005230B60F7BDC0461C
:102A600004E100E0AC020010A44004400C800040EF
:102A7000A84004408080044098800440788004404E
:102A8000A404001028800040048000400080004022
:102A9000088000401480004000E100E008B5FFF726
:102AA0007FFFC268031C1202120E8218D07BDA6804
:102AB0001202120E0132D2B29A7352B2002A01DA15
:102AC00000229A7308BD10B5041CFFF769FFC268A5
:102AD0001204120E8218D473C2681204120E01324C
:102AE000D2B2427352B2002A01DA0022427310BD00
:102AF00008B5FFF755FFC268C36812021B041B0E1E
:102B0000120ED01A431E9841C0B208BD70B5002401
:102B10001D5D0619002D02D005550134F8E7121B82
:102B2000301C131C002B03DD0170013B0130F9E761
:102B3000D043C0170240A01870BDF7B5051C019125
:102B40000093561E092B01D8041C0CE000980A21A2
:102B500002F022FE0199031C321C281CFFF7EDFF36
:102B6000071C2C1807E0671B002E04DD019B013EAB
:102B700023700134F7E700980A2102F051FE30314A
:102B8000781C2170FEBDF8B50C1CD9175F18051C08
:102B90004F40561E092F12D9381C0A21002B03DA88
:102BA00002F0FAFD434202E002F0F6FD031C281C8D
:102BB000211C321CFFF7E7FF041C2D1814E0002B2A
:102BC00000DA961E2A1CA919891A002902DD147040
:102BD0000132F8E7F443E41734402D19002B03DAEF
:102BE0002D232B7001340135381C0A2102F018FE08
:102BF00030312970601CF8BDF7B5089F1E1C051CFC
:102C0000013A3B0901D1041C05E00093331CFFF796
:102C1000F3FF2C1806E0601B002A03DD2170013A47
:102C20000134F8E70F231F40092F01D8303704E0A3
:102C3000002E01D0373700E0573727700130FEBD36
:102C4000F0B585B0041C029101D00021017000256F
:102C50001178002906D1029F0023BD426CD2237057
:102C6000281C6FE0029FBD42F5D2252902D0013217
:102C7000217004E05178252904D1217002320135F8
:102C80000134E5E7302902D0561C202100E0961CD3
:102C900032782D3A50424241B6180022307830271F
:102CA0007F423F18FFB2092F07D80A277A438218BC
:102CB000D2B2303AD2B20136F0E7AF18BC46029F2A
:102CC000BC4501D97A1BD2B2692818D00BD8632829
:102CD0002AD0642813D0582832D11F1D1B68201C0D
:102CE000009301231DE075280FD0782814D0732895
:102CF00026D11F1D201C1B68FFF708FF0AE01F1DBF
:102D0000201C1B68FFF73FFF04E01F1D201C1B68F1
:102D1000FFF713FF3B1C0BE01F1D1B68201C0093DB
:102D20000023FFF769FFF5E71868043320700120DE
:102D3000721C24182D188BE7013C2370681E01E0DB
:102D40000120404205B0F0BD10B50C1C131C6421DD
:102D5000221CFFF775FF10BD00B5031C9BB00A1CB9
:102D600001A8191CFFF7F0FF632800DDFEE701A8AA
:102D700000F0B6F81BB000BD0FB407B504A908C930
:102D8000181C0191FFF7E8FF03B008BC04B0184716
:102D90000EB403B503AA08CA191C0192FFF7D4FFA9
:102DA00002B008BC03B0184730B50C1C0443032321
:102DB0002340041C002B01D0002310E0032AFBD980
:102DC000CC58C4500433D41A032CF9D8131F9B08D1
:102DD00001339B00C418C91803231A40ECE793423F
:102DE00003D0CD5CE5540133F9E730BD30B5031CA9
:102DF000840701D1032A01D89A1814E00B060C04A9
:102E00001D1C25430D430C022543031C20C38418BD
:102E1000E41A032CFAD8131F9B0801339B000324E8
:102E2000C3182240E8E7934202D019700133FAE751
:102E300030BD021C031C981A0133591E0978002961
:102E4000F9D17047031C0A781A70002A02D00131A8
:102E50000133F8E7704730B50023934208D0C45CD3
:102E6000CD5C651B06D10133002CF6D1201C02E09D
:102E7000002000E0281C30BD10B50022835C8C5C73
:102E8000A34204D10132002BF8D1181C00E0181B1A
:102E900010BD000008B5094BFA211868890002F03E
:102EA000C9FCFFF745FB96200002FFF77DFD0120DE
:102EB000FDF7C8F9FEF72AFF08BDC046A4040010BC
:102EC00008B5FEF7ABFFFFF7EFF8FFF797F9FEF74E
:102ED00065FBFEF751FBFFF7DDFFFFF7DDF808BDEF
:102EE00010B5041C2078002803D00134FDF7FAF94E
:102EF000F8E710BD38B5051C0E24013C04D3295D4C
:102F00000248FFF739FFF8E738BDC046A46B000060
:102F100038B51948FFF730FF184C201CFFF7EAFFBF
:102F2000174D4221281CFFF727FF201C0E30FFF70A
:102F3000E1FF4321281CFFF71FFF201C1C30FFF777
:102F4000D9FF1048FFF718FF201C4630FFF7D2FFCB
:102F50000D48FFF711FF201C2A30FFF7CBFF281C7C
:102F60004E21FFF709FF201C3830FFF7C3FF616DCA
:102F70000648FFF701FF38BDA76B0000E004001012
:102F8000AD6B0000B46B0000BA6B0000C06B0000BA
:102F900003110A2253430F2210401818704738B506
:102FA0000A21041C02F046FC0A210501201C02F043
:102FB00097FC281C084338BD08B5C12252000E20DA
:102FC0000221FEF7FDFD024B01225A7108BDC046E9
:102FD000D404001010B5084C6379002B01D1FFF721
:102FE000EBFF23790C221A43A37901205B001A43DB
:102FF000011CFEF7E5FD10BDD404001010B5074C10
:103000002379002B08D16379002B01D1FFF7D4FF7E
:1030100001232371FFF7DEFF10BDC046D40400106A
:1030200008B5054B1A79002A05D000221A711A72C8
:10303000DA70FFF7CFFF08BDD404001010B50121EE
:103040000220FEF7FBFD064B041C18787F23184076
:10305000FFF79EFF034B5870DC71201C10BDC0466B
:10306000B0040010D4040010014B01229A70704784
:10307000D4040010024B00229A701A727047C046A6
:10308000D404001008B5FFF7D9FF094B094A997815
:10309000002908D0197A012901D8013103E010680C
:1030A0000549086000E019720021D970116008BD5F
:1030B000D4040010740200107802001008B5FEF766
:1030C00003FE0C23184003D0024B1A7810431870EB
:1030D00008BDC046D404001010B5FFF7EFFF054B44
:1030E0001A781C1C530701D5FFF7CCFF002323706F
:1030F00010BDC046D404001008B50020FEF7CAFB7E
:10310000002801D0FFF7E8FF08BD000010B5054C0E
:103110000023E371FFF7F0FFE379002B01D1FFF704
:103120008DFF10BDD404001008B50948092102F034
:10313000E3FB084BFA22D2001A80FFF7E7FF064BA9
:1031400000221A60FA22054B92001A6008BDC046A0
:10315000D4040010DE040010740200107802001085
:1031600008B5FFF7C9FF002008BD08B5FFF758FFF5
:1031700008BD000070B51D4C061C637822781B0248
:103180001343A278A07912041343E2780D1C1206AF
:103190001343174A13401A0A237062701A0C1B0E4D
:1031A000E3706379A27022791B021343114A134022
:1031B00023711B0A6371FFF7EBFE0F4B1B88C018CE
:1031C00030806079FFF7E4FEB070E078FFF7E0FE52
:1031D000F070A078FFF7DCFE28706078FFF7D8FE6B
:1031E00068702078FFF7D4FEA87070BDB00400109E
:1031F0007F7F3F3F071F0000DE040010F0B58DB059
:10320000051CFEF72BFD002804D1281C1249FFF7EE
:10321000BFFD1EE00AAE0BAC211C301CFFF7AAFF5D
:103220003388F7780793B378267808936378A4787F
:1032300009930A4B187900F0D7F8099B0490029380
:10324000009701960394281C0549079A089BFFF7ED
:103250009FFD0DB0F0BDC046CC6B0000B004001067
:10326000D16B000070B5061C0D1C141CFEF7F6FC9B
:1032700000280AD0301C291CFFF77CFF002C07D047
:10328000044B00201B79236003E00120404200E052
:10329000201C70BDB0040010F7B504880E1C051C7E
:1032A0006421201C0092019302F0BAFA114B8FB2F4
:1032B000B078E41B1C80FFF772FE0F4CA070707892
:1032C000FFF76DFEE0703078FFF769FE2071E87857
:1032D000FFF765FE009B6071A371A878FFF75FFEA2
:1032E000E071381CFFF75BFE20720198FEF7C8FC06
:1032F000FEBDC046DE040010C004001008B5022365
:10330000FFF7CAFF08BD08B5021C501E82415201DA
:1033100000200121FEF754FC08BD38B5041C012033
:103320000D1CFFF7F0FF201C00F086F8072102F0CB
:10333000D7FA201C0A1C291CFFF7E0FF962040004A
:10334000FFF710F90020FFF7DEFF38BD73B5041C4E
:10335000FFF774FE002801D100203BE01E4B5D7892
:103360001E1C7378AB4207D10A20FFF7FBF8FFF76A
:1033700065FE0028F5D1EFE7FEF770FC0028EBD0E2
:1033800001A96846FFF7F6FE684600F055F8051CEF
:1033900001A800F031F8114B04199C420DD9E31734
:1033A00001221343ED18281C694600F075F8002C23
:1033B00001DA0B4B00E00B4BE418201C01A900F0D4
:1033C00024F8281C072102F08BFA68460A1C01A980
:1033D000FFF794FF76BDC046D40400107F51010072
:1033E0008051010080AEFEFF07231840014B800092
:1033F000C0587047446C000002783C235A4341781F
:103400005218534382789818704738B50C1C3C21E9
:10341000051C02F065FA281CA1703C2102F00AFA92
:103420003C2102F05DFA6170E121281C090102F0E3
:1034300001FA207038BD000070B5837802210022A7
:1034400099425241048896214901051C64180C20B8
:10345000A41A42439B18033B99205843052102308C
:1034600002F0E8F96E26FF3666436421A310861940
:103470004942201CF61802F0DDF9C821361849002F
:10348000201C02F0D7F9034B3018C018EB78C01895
:1034900070BDC046D382FFFFF8B5204B0C1CC51889
:1034A0001F4B8000C0181F4902F0C4F90323584382
:1034B000C617B60F3618B610AE19B600953E301CBA
:1034C000194902F00DFACD17AD0F6D180527AD1093
:1034D0007D430235281C992102F002FA081C391C90
:1034E00002F0A8F90130E0709921281C02F0A2F93D
:1034F0000C21023002F0F4F94D1CEDB2A570301C25
:10350000094902F097F9094B0C21C6180E20401BFF
:1035100002F090F936182680F8BDC0467905000003
:10352000652F0400B13A0200B505000094EDFFFFDD
:10353000012008B5011C021CFEF714FE0120021C2C
:103540000221FEF70FFE0120011C0022FEF7BAFD4A
:10355000012002210022FEF7B5FD0120FFF78EF9C0
:1035600008BD0000194B70B50D1C19680722914366
:1035700019601968012421431960154B061C19684C
:10358000201C914319601A68211C22431A60221CD6
:10359000FEF798FD221C201C0221FEF793FD0D4B27
:1035A000311C186802F046F9011C201CFFF786F94F
:1035B000201CFFF773F9084E201C3560FFF74EF909
:1035C0003368002BFCD1FFF7B3FF70BD7C40044093
:1035D00080400440A4040010A0020010F8238A01D7
:1035E000DB0013404A05920E1343F82212021140E9
:1035F00019430A23594330B5CA1083181C1CEB34F5
:103600005D782478EA336C401B7824021C43835C89
:10361000201C58400723194008418005800D30BD0B
:103620007047000008B5054B011E994201DD044BAF
:10363000C1180448EA38FFF7D1FF08BDFF170000A2
:1036400000F8FFFF806C00000723594310B5084BBA
:1036500059189C310023CC5C0F2222400270CA5CB6
:103660000133120942700230072BF4D110BDC0465D
:10367000E00400100723594310B5074B59189C313B
:1036800000234278047812012243CA5401330230E5
:10369000072BF6D110BDC046E004001070B5AC4C4D
:1036A00086B0E36E6E465A1E934117363370A94BAF
:1036B000E258D006400F0138062807D802F058F823
:1036C000040C2012181A1D00022509E0636E16333F
:1036D0009B001B591D1C15E0636E16339B00E558BB
:1036E00000230FE0A36DE56DAB420BDD0D2509E076
:1036F000022503E00C25032304E00D252B1C01E02B
:103700000D25EDE750111F2800D91BE102F03AF812
:103710002000220029002C002F0033003B00440031
:1037200048004C00540061006E00760083008F005A
:103730009B00A800B800C500D500D300E100E4005C
:10374000E700EF00FE0002010B010D010F01150162
:10375000E01801E0E0180E30EB1A591C02F0CCF82A
:10376000F0E0E0181C30F7E7211C0E3105E0E0180E
:103770000E30E1180BE0211C1C31201C1A1C2B1CE4
:1037800001F08DFADEE0E018E1181C300E31EB1A82
:103790005A1CFFF709FBD5E06F48011C0E31EDE71D
:1037A000E018011C1C31F2E7226E1021002A00D023
:1037B0000A21221C0E3206E0226E1021002A00D0BF
:1037C0000A21221C1C32029100950196201C211C0A
:1037D00053E0216E012232701022002900D00A220B
:1037E000009501960292201C211C45E0226E1021BA
:1037F000002A00D00A21221C0E3213E0216E012281
:1038000032701022002900D00A22009501960292FF
:10381000201C211C4DE0226E1021002A00D00A211C
:10382000221C1C32009501960291201C6AE0226E37
:103830001021002A00D00A21484A029100950196E1
:10384000101C111C19E0216E1020002900D00A2044
:10385000424A0290111C1C3900950196101C0CE084
:10386000216E012232701022002900D00A223B4929
:10387000009501960292081C002201F01AFA61E0FC
:10388000226E1020002A00D00A20344A0290111C17
:103890001C3900950196101C35E0216E0122327012
:1038A0001022002900D00A222C490095019602928C
:1038B000081C002227E001223270226E1021002A0B
:1038C00000D00A21254A029100950196101C002182
:1038D00019E0009620481BE00096204818E0226E70
:1038E0001021002A00D00A21221C1C3206E0226E80
:1038F0001021002A00D00A21221C0E3200950196C8
:1039000002910020211C01F0FCF91BE00096201C14
:10391000002103E0211C1C310096201C1A1C2B1CCA
:1039200001F052FA0EE0201C02E00B4800E00B48C8
:10393000191C2A1C01F05FFA04E0201C191C2A1C27
:1039400001F063FA33780120E36606B070BDC0462B
:10395000E0040010C4070000EE040010FC04001096
:10396000064B10B51A1DD46F191C0831CC67D96FDE
:10397000D1679A6F9867DA6710BDC046E0040010FF
:10398000064BD96F1A1D986F9967D16F0833596725
:10399000D96FD1670022DA677047C046E004001093
:1039A000F8B5134C261C8C3630680130FFF73AFE10
:1039B000F923DB00E0500F4B0122E758A36E051CF2
:1039C00002409A4211D1830703D430680230FFF7D6
:1039D000C7FFFF2292001540231CAD01BF108C339E
:1039E0002F431F60044B0122E2500220F8BDC04665
:1039F000E0040010C4070000AC0700000F4A104BA1
:103A000030B5D158131C8C331C68CB059B0E01209C
:103A10008D0501D5403B02E0002B00D1031C89102D
:103A20000840916E884206D1111C8C31E3180B605E
:103A3000044B0121D150012030BDC046E0040010EC
:103A4000C4070000AC07000008B5084B5A1CD07F23
:103A50009A1CD27F00011202104303331A7FDB7FCE
:103A600010431B031843FFF77BFF08BDE004001061
:103A700008B5FFF785FF0323044A0F219A18014078
:103A8000013311770011072BF6D108BDE0040010B7
:103A900008B5FFF775FF044B01211A1C8C3210602A
:103AA000024A995008BDC046E0040010AC0700006F
:103AB00010B5064CA36E002B07D0FFF761FF231C47
:103AC0008C331860024B0122E25010BDE00400105C
:103AD000AC07000010B5064CA36E002B07D1FFF712
:103AE0004FFF231C8C331860024B0122E25010BDA3
:103AF000E0040010AC07000008B5054A054B0121A1
:103B0000D150054B1B68002B00D0984708BDC0461C
:103B1000E0040010BC0700003C03001038B5154A53
:103B2000154B00209850F822D2009A5882421AD0A1
:103B3000F622D200995881421ADD012909D1F721D4
:103B4000C9005C58844204D00C4D58500A215C5185
:103B500099509A58032A01DD0121D966F621013ACC
:103B6000C9005A5004E0064B1B68002B00D0984750
:103B700038BDC046BC070000E0040010B4070000D8
:103B80003C030010094BF822D2009A58002A04D0B6
:103B9000F622D2009A58002A07DD054A0F219A58CA
:103BA0000133114099771211DA777047E004001061
:103BB000B4070000044B597F9A7F090112020A439F
:103BC000197F0A435A677047E00400100B1C093B39
:103BD00030B5012B0FD80023074A9C18257FC45C01
:103BE000A54205D0054B0839D0580143D15002E019
:103BF00001330E2BF0D130BDE0040010A40700000B
:103C000008B508290DD0192913D1427808231A4282
:103C100002D00022027002E00F23037007234370DA
:103C200005E000230022C25401330E2BFAD1FFF726
:103C300021FD08BD30B5114D85B06C6F002802D054
:103C40000F239C4304436C67FF2C05DD281C1C30AC
:103C50000E2101F051FE0FE06846211CFFF7F4FC35
:103C60006846211CFFF7CCFF00236846C15CEA18B8
:103C7000013311770E2BF8D105B030BDE0040010F0
:103C8000134B30B5596F0F229143041C0C4385B080
:103C90005C671D1C082C19D0FF2C17DC6846211C02
:103CA000FFF7D2FC6846211CFFF790FF0023EA18BB
:103CB000127F6946CA5401330E2BF8D16846211C85
:103CC000FFF79EFF6846211CFFF7D4FC05B030BD0E
:103CD000E00400101FB50F4C616F082918D0FF29B0
:103CE00016DC6846FFF7B0FC6846616FFFF76EFFB1
:103CF0000023E218127F6946CA5401330E2BF8D113
:103D00006846616FFFF77CFF616F6846FFF7B2FCA2
:103D10001FBDC046E004001010B50D4C631CD87FD9
:103D2000A31CDB7F00011B021843E37F1843E31C45
:103D3000DB7F1B031843FFF775FC0F23021C1A409F
:103D400022770211134000126377A07710BDC0469E
:103D5000E0040010044B5A6E16329200D258121A28
:103D600051424A41DA667047E0040010044B5A6E33
:103D700016329200D158013900D50D21D15070472B
:103D8000E0040010054B5A6E16329200D1580131F2
:103D90000E2900D10021D1507047C046E004001028
:103DA000144B10B55A6E191C16329200D2580C2AB8
:103DB00005DC9A18507F117F0001021C17E00E48A5
:103DC000F5241858A400A04205D00C4C2040B7247C
:103DD000A400A04207D18A18137F486D1B0102116D
:103DE00013434B6505E09A18127F197F12010A43AD
:103DF0005A6510BDE0040010CC070000FFFEFFFF75
:103E0000264B10B55A6E16329200D2580C2A05D1A4
:103E100023495858F5218900884204D0FA21C90065
:103E2000595800290DD0596D0F240C409A180811CB
:103E3000107754770901FF22114008431C77586519
:103E40002BE00C2A07DC596D9B180F220A40091140
:103E50001A77597721E0124AF5219A5889008A4247
:103E600005D010490A40B72189008A420DD15A6D08
:103E70000F20191C1040293108701001FF21084043
:103E80001111021C0A435A6507E05A6D191C1011E2
:103E9000293108700F210A401A7710BDE004001084
:103EA000CC070000FFFEFFFF244B0F215A6E586D18
:103EB00016329200D258014070B500110C2A05D17B
:103EC0001F4C1D59F524A400A54204D0FA24E40097
:103ED0001C59002C09D09C18657F267F2D01354385
:103EE0005D651D7F2077657726E00C2A08DC9C182D
:103EF000657F267F2D0135435D65607721771CE066
:103F00000F4AF5249A58A400A24205D00D4C224035
:103F1000B724A400A24207D11A1C293214781170C8
:103F200024012043586508E01A1C293214781D7FAB
:103F300024012C435C651070197770BDE0040010FB
:103F4000CC070000FFFEFFFF08B503480E22011C4E
:103F50001C39FEF729FF08BD1805001008B50348F5
:103F60000E22011C1C31FEF71FFF08BDFC040010CF
:103F700008B504480022011C1C310D2300F08FFEFF
:103F800008BDC046FC04001008B503480E22011C01
:103F90000E39FEF709FF08BD0A05001008B50348F1
:103FA0000E22011C0E31FEF7FFFE08BDFC040010BE
:103FB00008B504480022011C0E310D2300F06FFEED
:103FC00008BDC046FC0400100023044A00219A18D2
:103FD000463201331170082BF7D17047E00400100E
:103FE000C31C421E0020934207D0044940005918C8
:103FF00046310978013B0843F5E77047E0040010BB
:1040000010B50B1D994208D0044A01248A180440B7
:104010004632147040100131F4E710BDE004001086
:1040200038B50020FFF7DCFF084C051C0021207F7D
:10403000FFF7E6FF04202577FFF7D2FF0421051CD8
:10404000607FFFF7DDFF657738BDC046E0040010F4
:1040500010B50020FFF7C4FF034C20770420FFF7C2
:10406000BFFF607710BDC046E004001010B5054CDE
:104070000021207FFFF7C4FF607F0421FFF7C0FF0E
:1040800010BDC046E004001010B50A4C231C8C3350
:1040900018680130FFF7C6FAF923DB00E050021C74
:1040A0000F231A4022770211134000126377A07782
:1040B00010BDC046E004001010B5084C0E21201CB5
:1040C00001F01AFC201C0E300E2101F015FC201C02
:1040D0001C300E2101F010FC10BDC046E0040010A1
:1040E000054B1A1C0E32197F187801330143D9761B
:1040F0009342F8D17047C046E0040010054B1A1CEB
:104100000E32187F197801330140D9769342F8D1E5
:104110007047C046E004001030B5002185B00E4B5A
:10412000421C1818007F6C4608550D25D40F181C2A
:10413000002395425C416442013122400E2901D0A6
:10414000101CECE76C46E15CC218013311770E2BB2
:10415000F8D105B030BDC046E0040010074B10B5E3
:104160005A6E16329200D458611E1C19D150207715
:10417000002901DA0D21D15010BDC046E004001025
:10418000034A0023111C943198320B60136070476E
:10419000E0040010034B0122943319684A401A606E
:1041A0007047C046E0040010074B0022191C8C31F8
:1041B0000A601A67054A012199501A1C9432126844
:1041C00051424A41DA667047E0040010AC07000033
:1041D0009A4B9B4910B5CC580F20A310994A184010
:1041E000A411013812570E2844D801F0C1FA080E64
:1041F000151C20432643432D434343313500002AF9
:1042000038DB8A184032002304E0002A32DB8A18A7
:104210004032012393712BE0002A2BDB8A184032B5
:104220009379CB6624E0201CFFF798FF20E0002A5A
:1042300020DB101CFFF78EFD1AE0002A1ADB4B6E04
:1042400016339B00CA5013E0201CFFF719FD0FE046
:10425000201CFFF7EFFC0BE0002A0BDB101CFFF724
:104260005BFF05E00C2B20DD162B25D1FFF798FD19
:104270000120E9E0982B02D100230B66F8E7982B88
:1042800069DC382B02D101204866DDE0382B2EDCBA
:104290001C2B02D1FFF758FEEAE71C2B11DC0C2B7C
:1042A000E0D1983101200860CEE00120002B00D140
:1042B000CAE001204042C7E0182BFAD1FFF774FF93
:1042C000D6E7282B02D100234B66D1E7282B04DC4C
:1042D000262BEED1FFF794FDCAE72C2B02D1FFF776
:1042E0003DFEC5E7362BE4D1FFF7DEFDC0E7662BC8
:1042F00002D1FFF753FEBBE7662B16DC4C2B03D134
:10430000FFF7C2FE02209FE04C2B04DC3C2BD0D1F7
:10431000FFF72EFEACE7562B02D1FFF735FEA7E7DD
:104320005C2BC6D1FFF790FBA2E76C2B02D1FFF705
:104330009FFB9DE76C2B04DC682BBAD1FFF7BCFE1A
:1043400096E7762B02D1FFF733FE91E7882BB0D1A9
:10435000FFF718FC8CE7E62B02D1FFF779FE87E721
:10436000E62B33DCC82B02D1FFF714FF80E7C82B04
:1043700015DCA82B02D10120086665E0A82B04DC1F
:104380009C2B96D1FFF716FC72E7B82B02D1FFF7F2
:10439000F7FE6DE7BC2B8CD1FFF79CFC68E7D62BB2
:1043A00002D1FFF763FE63E7D62B04DCCC2B80D170
:1043B000FFF7B2FC5CE7D82B02D1FFF779FB57E798
:1043C000DC2B00D075E7FFF78BFE51E7F32B02D112
:1043D000FFF7A4FB4CE7F32B17DCEC2B02D1FFF724
:1043E0008DFE45E7EC2B05DCE82B00D061E7FFF7FD
:1043F00071FB3DE7F12B02D1FFF7E6FD38E7F22B29
:1044000000D056E7FFF778FB32E7F62B02D1FFF733
:1044100007FE2DE7F62B05DCF52B00D049E7FFF76B
:10442000A5FC25E7F72B02D1FFF7ACFC20E7F82B22
:1044300000D03EE7FFF72CFB1AE7C046C407000098
:10444000E004001080A8000010BDC04638B51E4C26
:104450001E4D1F4B6159E150231C8C331868FFF728
:10446000E1F8E26E1B4BA2660022E266E2500322F4
:10447000605110401D1C022809D090420AD001282A
:1044800002D0FFF7A5FE07E0FFF78AFA04E0FFF786
:1044900005F901E0FFF7B2FA00280CDD6359002BA3
:1044A00004D1231C8C3319680A181A60231C90331A
:1044B00019680A181A60FA23DB00E258002A01D0B2
:1044C000013AE25038BDC046E0040010C4070000C5
:1044D000CC070000AC070000034B0122DA660F2274
:1044E0009A775A771A777047E004001070B5084C35
:1044F000F425ED006659201C064901F0FDF96651CE
:10450000FFF7EAFF044A01236366A35470BDC04667
:10451000E0040010D40700009C0700007047000072
:1045200030B50D4D049C28600C4801600C490A60B0
:104530000C4A13600C4B039A1A600C4B0C4A1C601B
:10454000F423DB00D4500B4A0B4B1A600B4B0C4A84
:1045500013600C4A136030BD68030010780300102C
:10456000840300104C0300104403001018000010D6
:10457000E0040010A54600003C0300101D450000AB
:104580007C03001060030010014B18607047C046A8
:1045900048030010094B10B51A68191C084B002A73
:1045A00003D1084C2468226003E01A68904200DAC4
:1045B000101C186001230B6010BDC0465003001092
:1045C0007403001048030010034B1B68002B01D13B
:1045D000024A13607047C0465C030010500300108D
:1045E000014B4A3318787047E004001070B5194D3C
:1045F0002B1C98331B68002B04D0174B1C6801231D
:104600001C4002E02B1C94331C68F523DB00EB58A4
:104610009C4203D1114AAA58002A19D0002C02D179
:10462000002B0BD114E00E4B0C4E1B68002B02D05C
:10463000201CA95998470023AB5106E0084B1B6882
:10464000002B02D0201C211C9847F523DB00EC50E6
:1046500070BDC046E004001058030010A40700001D
:1046600068030010084B1860084B196000280AD036
:10467000074A01231370074A00211170064A0749AF
:104680008850074A13707047640300106C030010D1
:104690008003001054030010B4070000E004001071
:1046A000400300102D4B73B51A682D4B1168186824
:1046B00081421BD000210091019112681A60294BA0
:1046C0001B688B4202D0684601A99847264B009987
:1046D0001C68181C019A254BA14202D11C68A242F9
:1046E00002D0234C0125257001601A60214D224B18
:1046F000EB58002B10D01E490023CB56002B2CD09A
:104700001E4B00229A56012A27D100220A701C490A
:104710000A7002221A7020E0134B184C1868002807
:1047200007D00023E356002B03D1104B1968FFF785
:1047300099FF0023E356124E022B04D1114A0023A5
:104740003370AB5023700023E356002B02D00A20B5
:10475000FFF720FF0023F356EB6673BD4C030010F8
:104760001400001078030010640300106C030010A4
:1047700054030010E0040010BC07000040030010C8
:1047800080030010B407000038B5064CF823DB00A6
:10479000E358002B05D1E56E034AA350FFF782FFD3
:1047A000E56638BDE0040010BC07000008B5084A03
:1047B000084B126819688A1A05D5FA2252001A6045
:1047C000054B1A6801321A60FFF710FF08BDC0469A
:1047D000440300101C0000105803001037B5041CDF
:1047E0000025002300930193124B1B68002B02D07D
:1047F000684601A9984700980135002800D0002597
:104800000220FBF7CBFD0C4B1A680C4B11681868A3
:1048100081420AD012681A60FFF7C8FF002C04D04A
:10482000013C002C01D1201C02E0032DD9DD012028
:104830003EBDC046780300104C030010700300100A
:10484000F8B50E1C0E21041C171C01F055F8174B6F
:1048500003259E4211DD092363730123237323E0A3
:10486000301C0A2101F03CF8301C61550A2100F08F
:10487000E1FF0135061C0D2D01D0002EF0D1EF1BFC
:10488000033F27706B1E022B05D0E15C621BD21820
:104890005173013BF7E70F235D1B013D6B1C032B9D
:1048A00002DD00236355F8E7F8BDC046FFC99A3B17
:1048B0000278002A01D1802252004378002B01D1D6
:1048C00080235B00D01A7047F0B59B23234D5B001B
:1048D000EC5C85B003900E1C002C01D18024640098
:1048E0003023FF33EB5C002B01D180235B0002936C
:1048F0003823FF33EA5C80235B009C4203D00F2304
:10490000171C1F4000E007271548FFF7D1FF029949
:10491000421C631A802149000C1B0721C91B00940B
:10492000019103980F49FEF733FA002333704124B5
:10493000301CFEF77EFABA235B003718E818001B1C
:10494000FFF7B6FF221C031C0749381C0134FEF791
:104950001FFA462CECD105B0F0BDC046E0040010B3
:104960001406001090A800009DA80000F0B5F722E2
:10497000734CD200A150221C9432724B126895B035
:10498000051C0E1CE050002A1AD118280BD1C3298F
:1049900009D16D4B1B680F2B05D1201C38300E211F
:1049A000162200F067F967482058182806D1F72327
:1049B000DB00E358332B01D100F0F6F8FFF78CFD54
:1049C000F623DB00002D02D00A22E25000E0E55081
:1049D000281C311CFFF746FE5C4D5D4E2B681B68A2
:1049E0003360FFF7F1FD012323671E2200230292AB
:1049F0000393584B1B68002B1AD0574D2B682F1C64
:104A0000002B15D01B68002B04D1544B1B68984712
:104A10003B68F7E72B681A68013A1A60504A136836
:104A2000002B05DD013B1360002B01D1FFF7CCFD0E
:104A3000FFF70CFD002809DA231C8C331A680132B9
:104A40001A60231C90331A6801321A60454B039890
:104A5000454D98420CD04023021C9A43434B9A4246
:104A600006D0434B984203D0F3239B00984211D1C8
:104A70006359404A93420AD02022191C91433E4A6E
:104A8000914204D0402293433C4A934202D10A20EF
:104A9000FFF780FD65593A4A0395251C8C352B6834
:104AA00093421BD0374A93420FD0374A934224D1C6
:104AB000FFF79CFDFBF7A2FC344B224A18603368D9
:104AC000A050013B3360324B16E0324B1B68002B89
:104AD00013D0314A0120A15898470EE02F4F3B6870
:104AE000002B0AD004A80CA9FFF7EEFE3B6804A82F
:104AF0000CA998472B6827332B60029D0298013D33
:104B0000002813DC264B1E251B6898470F4B1A689C
:104B1000244B11681868814208D012681A60FFF7A8
:104B200033FEFFF743FE0D4B1B689847226F002AA8
:104B300001D002955DE7FFF759FD15B0F0BDC04605
:104B4000E0040010B4070000180000104C0300102F
:104B50001400001050030010480300107C030010E4
:104B6000740300106E020000C4070000260200005B
:104B70007A020000FB030000CB030000A303000047
:104B80003E2700005C280000790D0000640300103F
:104B90007E0D000068030010A407000084030010CD
:104BA0006003001070030010F7B52C4D00202B6837
:104BB0001C68FFF713FE2B681A689442FCD01B6830
:104BC000274E2D33FF330193FFF786FC254CF62348
:104BD0000A22DB00E2501823A351F7231522DB0041
:104BE000E250F8230127DB00E750231C903300221A
:104BF0001A60FFF771FC27672B68019A1B689A42BD
:104C00000CD0FFF723FC2A68174B11681868814203
:104C1000F2D012681A60FFF7C9FDEDE7231C90334C
:104C20001D68F823DF00012618200021E651FFF758
:104C30009DFE0E4B281C196800F0FCFD0422011C8F
:104C40000B48FFF7FDFD064818232350F7230022E9
:104C5000DB00E651281CE250FEBDC0464C030010AC
:104C6000B4070000E00400107003001044030010BB
:104C70001805001070B5002A10DD047801231C40CF
:104C80004B1E002B08DBC55CE4006E083443C454A3
:104C90000124013B2C40F4E7013AECE770BD30B54C
:104CA0009A4205DC845C8D5C85548C540132F7E7B4
:104CB00030BDF0B5069E051C07A804783078002AA0
:104CC00017D0059EB34217DCCE5CD75CF7193F18AE
:104CD0000020A74201DB3F1B0120EF540133F0E726
:104CE000CA5C12180020A24201DB121B0120EA5408
:104CF0000133059A9342F3DD01231840069B187097
:104D0000F0BDF7B50AAC2478099D0094089E2C7874
:104D1000002833D000292ED0002A1CD0B3424EDC0C
:104D2000CF5CD55C7F1B3F1B0024A74204DA009CAC
:104D30003F190F2427400124C7540133EEE7CA5C12
:104D4000121B0024551C04D1009C0F22013C224060
:104D50000124C2540133B342F1DD30E0D15C494259
:104D6000091B0024A14204D0009F0F24C91921402F
:104D70000124C1540133B342F0DD20E0002914D0F6
:104D8000002A08D0B3421ADCCD5CD05C0133281A6B
:104D9000041BE40FF6E7B34211DCCA5C0133141BB9
:104DA000013462425441E4B2F5E7B34207DCD15C1E
:104DB000013349420C1B611E8C41E4B2F5E701232B
:104DC0001C40099B1C70F7BD70B5049C0125257023
:104DD00000290BD09A420BDC865C8D5CAE4209D177
:104DE0000132F7E7815C002904D101329A42F9DDF2
:104DF0000023237070BD914204DA43185B7843545A
:104E00000131F8E70023435470478A4205DD8318D7
:104E1000013B1B788354013AF7E700238354704722
:104E2000F7B5134A134C13785278C35C134000D083
:104E30004023114923601231009100220023A6185B
:104E40007360009B0125123B1F785978C75D39427A
:104E500002D077682F437760009F02336D00BB421A
:104E6000F2D1123304320093282AE7D10020FEBD8C
:104E70000C0100104C0E001058000010122330B529
:104E80004B43334A0131D318052251431A785C78D9
:104E9000825C144204D02F4A5F24521894705470DC
:104EA0009A78DC78825C144204D02A4A7C24521816
:104EB000533214701A795C79825C144204D0254A0A
:104EC0007C245218A33214709A79DC79825C1442E3
:104ED00007D0204C5F226418251CA235A1342A700B
:104EE00022701A7A5C7A825C144204D0194A7C24BB
:104EF0005218A03214709A7ADC7A825C144204D080
:104F0000144A7C245218503214701A7B5C7B825CE9
:104F1000144207D00F4C5F226418251C52355134BF
:104F20002A7022709A7BDC7B825C144204D0094A8E
:104F30002E245218A43214701A7C5B7C825C1342BB
:104F400004D0044B5918F43127230B70002030BDD6
:104F500058000010B80C0010F8B52E4D061C0027A4
:104F60002C1C281C20214F22FDF740FF002F04D0CD
:104F70002A1C7C2339322B7013702B1C4F330022D8
:104F800001371A705035052FEBD1211C2D233831F4
:104F90000B70211C37310B70A121A3706370490085
:104FA0005F2363544221FF316354A32149006254BB
:104FB000194A11785278715C0A4204D0221C53328B
:104FC0005234137023700024211C301C0134FFF76D
:104FD00055FF0A2CF8D10024104B114DE25C1B192F
:104FE000B15C58780F4A6300084201D0D15805E0FF
:104FF000D058FDF71EFF0C49091A0A31281C02344B
:1050000000F084FC122CE7D1281C084900F07EFC3B
:105010000520F8BDB80C00100C0100102000001095
:10502000F80D0010340000100E010010A5A80000BB
:10503000034B0020185642425041C0B218707047CE
:1050400088030010F0B5884C87B021680390019167
:10505000FCF792FA854B86481B7886495BB2864AF4
:10506000002B07D002235B42036006230B60012361
:105070005B4202E0092505600B6013607F4B181C42
:10508000DE30458806887E482D04354385421BD195
:10509000E33358781D78000228439D78DB782D048F
:1050A0001B0628431843774B98420DD1764C0A686B
:1050B00023687648033323600921754BFCF74AFBCC
:1050C0002368033B236095E22368052B05D0062B5C
:1050D00009D0042B0AD06E4A09E001235B42136019
:1050E0006C4B029304E06C49029101E06B4A02921E
:1050F00000236B4D009300990C244C43002900D1F0
:105100000124594B1868022800DCCFE0002305AACF
:1051100053702B687F210B405B2B71D02CDC232B31
:1051200000D19EE014DC062B53D006DC002B4ED0C1
:10513000022B00D0B6E0492394E01C2B00D18EE076
:10514000212B00D186E0072B00D0ABE0372283E093
:10515000402B6DD007DC392B6ED03F2B66D0382B1F
:1051600000D09FE072E0502B74D0542B79D04F2B9D
:1051700000D097E033226FE0732B69D014DC662BEC
:1051800040D008DC5E2B59D0622B68D05C2B00D05D
:1051900088E04F2260E06F2B3AD0712B52D06D2BFC
:1051A00000D07FE0352257E0792B49D007DC762B01
:1051B0004AD0772B3ED0742B74D148224CE07D2B03
:1051C00022D07F2B22D07C2B6CD1422244E02023A2
:1051D00048E031231370009A022A00DC20E22B1CE5
:1051E000083B1B680B40542B30D0032A00D117E238
:1051F0002B1C0C3B1B681940542900D010E225E001
:1052000032232FE034232DE036232BE0382329E00E
:1052100039231370009B062B00DC01E22B1F1B6857
:1052200047221940232900D0FAE115E0302319E084
:105230002D2317E0412315E0432313E0442311E01D
:1052400045230FE046230DE048230BE04C2203E00A
:10525000502307E0522305E005AB1A70E0E1552327
:1052600000E04E231370DBE11C01001088030010E6
:10527000780E0010B40C0010480E0010E00400106E
:105280003D001D1111444C8004000010ADA8000029
:10529000BC680000AC680000B46800009C680000B6
:1052A0004C0E00100438414241410191019B012BF9
:1052B00000D184E0022B00D1F7E0002B00D06EE19A
:1052C00029680123194206D0CC4AA01C1178C0B22B
:1052D0000522FCF7C9F92A68920709D5C74BE01DDA
:1052E0001968C0B20131C9B201220323FCF7BCF92D
:1052F00029680423194208D0C04AE01D1168C0B2D1
:105300000531C9B20122FCF7AFF92A68120709D5A5
:10531000BA4BA01C1968C0B20931C9B205220123D9
:10532000FCF7A2F92B68DB0609D5B44B601C1968A1
:10533000C0B20531C9B201220423FCF795F92968EE
:10534000890609D5AD4B601C1968C0B20131C9B2DC
:1053500001220323FCF788F92A68520609D5A74BD6
:10536000A01C1968C0B20431C9B205220123FCF7A0
:105370007BF92B68D90516D5A04FA14E3A68336842
:10538000E4B2D118201C09300A31C0B2C9B2FCF70E
:1053900057F9396833680A34C9180931E0B2C9B21B
:1053A000FCF74EF9FBE0190600D4F8E0934B093402
:1053B0001968E0B20931C9B202220123EDE02A687E
:1053C000019B1A4210D08D4EE7B2B81CC0B23178A2
:1053D0000522FCF749F9316803370131F8B2C9B247
:1053E0000322019BFCF740F929680222114208D0F0
:1053F000824BA01D1968C0B20131C9B20323FCF76A
:1054000033F92A6804231A4208D07C4AA01D116887
:10541000C0B20531C9B20222FCF726F92B681B077E
:1054200013D5764EE7B23168B81C0931C0B2C9B2A3
:1054300005220123FCF718F9316803370831F8B267
:10544000C9B203220123FCF70FF92968C90609D55F
:105450006A4B601C1968C0B20531C9B2022204232C
:10546000FCF702F92A68920609D5644B601C19689A
:10547000C0B20131C9B202220323FCF7F5F82B6850
:105480005B0667D55D4EE7B23168B81C0431C0B227
:10549000C9B205220123FCF7E7F83168033705316B
:1054A000F8B2C9B20322012352E02A68D20707D515
:1054B000524B601C1978C0B20722019BFCF7D4F84C
:1054C0002B680222134206D04C4BA01D1978C0B2A3
:1054D0000623FCF7C9F82968490709D5474BA01DE1
:1054E0001968C0B20431C9B202220623FCF7BCF825
:1054F0002A68120709D5414B601C1968C0B20831EF
:10550000C9B207220223FCF7AFF82B68DB0609D5E6
:105510003A4B601C1968C0B20431C9B2022206239A
:10552000FCF7A2F82968890607D5344B601C197866
:10553000C0B202220623FCF797F82A68520609D562
:105540002E4B601C1968C0B20431C9B20722022375
:10555000FCF78AF82B68D90515D5284F284E3A68EC
:105560003368E4B2D118201C02220A300831C0B2DC
:10557000C9B2131CFCF778F8396833680934C918C4
:10558000E0B2093106E0190609D51C4B0934196847
:10559000E0B208310222C9B2131CFCF765F8009A88
:1055A0000435013200920B2A00D0A4E5154B1B688C
:1055B000002B06D0144B15481A680021144BFCF739
:1055C000C9F8144D00240235AB1E1A7803996B1EDE
:1055D0008A5C1B78134209D00F4BA200D0580F4BA6
:1055E000E15C094B1A680A4BFCF7B4F80134023548
:1055F000092CE9D1FBF7CAFF07B0F0BDB40C0010CD
:10560000480E001054010010780E0010BCA80000D5
:10561000A4680000200000102001001013A9000061
:105620000C4E029B05A8211C3268FCF793F82B68EE
:10563000DA0506D5084B32681B68E11DD218074809
:1056400004E01A06ABD532680548E11D029BFCF761
:1056500081F8A4E7B40C0010480E0010BAA80000AE
:105660009069000038B5FEF7BBFF0624002805D17D
:10567000FBF78CFF38BD01340E2CF9DC0321201C14
:1056800000F0D8F80321C5B2201C00F029F9281C2D
:10569000C9B2FBF7D5FF092CEDD10B24EEE70000D2
:1056A00038B5041CFFF7BCFB201CFFF7CBFC094BF3
:1056B0001B78002B0DD0201CFFF74EFC064CC82396
:1056C0005B00E518211C05485034FDF755FBAC4242
:1056D000F8D138BD95030010B80C0010C75A00006F
:1056E00000B589B000280ED0FBF711FF01A80921F1
:1056F000FDF7AAFF684612300A21FDF7A5FF01A8B1
:10570000FFF7CEFF08E0FBF70AFF044B1B78002BE6
:1057100002D00348FDF730FB09B000BD950300102F
:10572000BEA80000FEE7FEE708B500230B4A0C49BF
:105730009A188A4204D20B49C95C01331170F5E70B
:10574000094B0A4A591C013B934203D200221A70AA
:105750000B1CF6E7FBF734FBFEE7C0460000001029
:10576000440100101CA90000450100107C0E00102F
:1057700002B4714649084900095C49008E4402BCE4
:105780007047C04603B47146490840004900095AB1
:1057900049008E4403BC7047002934D00123002205
:1057A00010B488422CD301242407A14204D28142A0
:1057B00002D209011B01F8E7E400A14204D28142B0
:1057C00002D249005B00F8E7884201D3401A1A432D
:1057D0004C08A04202D3001B5C0822438C08A04264
:1057E00002D3001B9C082243CC08A04202D3001B1A
:1057F000DC082243002803D01B0901D00909E3E794
:10580000101C10BC7047002801D00020C04307B412
:10581000024802A14018029003BDC046D900000012
:105820000029F0D003B5FFF7B9FF0EBC4243891A37
:105830001847C046002941D010B4041C4C40A4466F
:1058400001230022002900D54942002800D540420A
:1058500088422CD301242407A14204D2814202D2DF
:1058600009011B01F8E7E400A14204D2814202D2FF
:1058700049005B00F8E7884201D3401A1A434C08FC
:10588000A04202D3001B5C0822438C08A04202D332
:10589000001B9C082243CC08A04202D3001BDC085A
:1058A0002243002803D01B0901D00909E3E7101C9B
:1058B0006446002C00D5404210BC7047002806D03A
:1058C00003DB0020C043400801E08020000607B44D
:1058D000024802A14018029003BDC0461900000012
:1058E0000029EBD003B5FFF7A7FF0EBC4243891A8E
:1058F0001847C0467047C04642180023002903D00D
:10590000037001309042FBD17047C04670B5061C51
:10591000B30717D133680F480F4D1A189A43301C3C
:105920002A420FD1043002680A4BD41894432C4207
:1059300008D104300268074BD41894432C42F1D0AC
:1059400000E001300278002AFBD1FDF77BFA301C21
:1059500070BDC046FFFEFEFE808080805B4025302B
:105960003278253032785D0D0A0025732025730DBD
:105970000A00444D31355F4D314200534552494193
:105980004C20434F4E534F4C450072656164790083
:105990000D0A4279652E2E2E0D0A004E4F00203F33
:1059A000002573202573202025694D485A00563361
:1059B0003200202025692E253033695600202573BA
:1059C0005254432000524541445920464F522046EC
:1059D0004C415348494E4700444D3431204F4B0011
:1059E000424144204B4559202530327800202D205B
:1059F00025303278004C43443A25303269202D203E
:105A0000256900505245535320454E544552205469
:105A10004F20534156450053574953534D49435224
:105A20004F532028432920323031302D323032314B
:105A30000053495A453A256920555345443A25694A
:105A400020465245453A256900535441434B3A009C
:105A500025633120484F5552002D005254432052A7
:105A6000454144204641494C007475726E6564207E
:105A70006F6E003C52455345543E0D0A004261642E
:105A8000206E756D6265722E0D0A004241543A20F7
:105A900025696D560D0A000D0A2530327820200048
:105AA00057616974696E6720666F72206461746102
:105AB0002E2E2E0D0A00426164206D6F64656C0D00
:105AC0000A00526561642025730D0A004641494C65
:105AD0004544006F6666004C434420646562756708
:105AE0002025730D0A004B4244206F757470757445
:105AF0002025730D0A00436F6E736F6C6520746907
:105B00006D656F75742073657420746F202569202E
:105B10006D696E757465730D0A006F6E650074773C
:105B20006F0053617920626F6F746C6F616465728E
:105B3000202573206D6F72652074696D6525732053
:105B40002E2E2E0D0A004C61756E6368696E6720FB
:105B5000626F6F746C6F61646572202E2E2E0D0A59
:105B600000000000005C000C000C7C287C7C447C65
:105B7000241048285408000C003844004438002001
:105B80001008103810804000101010004000201045
:105B900008384438007C006454484454281C107C65
:105BA0004C542438542004740C28542808543800C9
:105BB00050008050001028442828284428100454FD
:105BC00008384C5C7814787C54283844447C443839
:105BD0007C54447C14043844347C107C007C0020C9
:105BE000403C7C106C7C40407C087C7C047C7C4489
:105BF0007C7C14083844787C1468485424047C0461
:105C00007C407C3C403C7C207C6C106C1C601C64A8
:105C1000544C7C4400081020447C00080408808018
:105C20008004080078447800040603000000007F28
:105C3000010704000007000000070B064400FF01F5
:105C400044004400FF014409058C009200FF0192CA
:105C500000620C06860046002000100088018401C6
:105C60000C06EE00110111012E01C00060010503B8
:105C70000000000007090500000000010182007C0F
:105C8000080400007C008200010109051000540096
:105C900038005400100905100010007C001000109E
:105CA00006030000800580030B06100010001000A2
:105CB000100010001006030000800180010905009B
:105CC00000C00030000C00030B06FE0001010101C2
:105CD00001010101FE0C06000004010201FF0100A8
:105CE0000100010C06820141012101210111010E77
:105CF000010B0682000101110111011101EE0B06D9
:105D00003000280024002200FF01200B068F00092C
:105D100001090109010901F10B06FC001201110141
:105D200011011101E00B0601000100E10111000960
:105D300000070B06EE001101110111011101EE0B1C
:105D4000060E0011011101110191007E06030000F1
:105D50009801980106030000980598030A051000B1
:105D600028004400820001010B06280028002800BA
:105D7000280028002809050101820044002800109D
:105D8000090502000100610111000E0B06FE000171
:105D900001190125012901BE0C06FE0111001100A7
:105DA00011001100FE010B06FF011101110111018B
:105DB0001101EE0B06FE000101010101010101824A
:105DC0000B06FF010101010101010101FE0C06FFAB
:105DD00001110111011101110101010B06FF011156
:105DE00000110011001100010B06FE00010101016C
:105DF00011011101F20C06FF01100010001000103B
:105E000000FF010A0501010101FF01010101010B70
:105E10000680000001000100010001FF0C06FF01E7
:105E2000100028004400820001010C06FF0100015F
:105E300000010001000100010C06FF010400180030
:105E400018000400FF010C06FF0104000800100008
:105E50002000FF010B06FE0001010101010101010B
:105E6000FE0B06FF0111001100110011000E0C06BF
:105E7000FE0001010101410181007E010C06FF01CC
:105E800011003100510091000E010B068E0011012E
:105E9000110111011101E2090501000100FF0101D9
:105EA00000010B06FF000001000100010001FF0BD3
:105EB000061F0060008001800160001F0C06FF01CA
:105EC0004000300030004000FF010C06C3012400F8
:105ED000180018002400C301090507000800F0019C
:105EE0000800070C06C10121011101090105010388
:105EF000010007080400000000BF01BF0109050000
:105F00000007000700070007130A00002000E40054
:105F1000FC003F00E700FC003F002700040F0800E2
:105F2000000C011E01FF03FF032201E201C2190D53
:105F300000000E001F0011019101FF007E00FC0017
:105F4000FE0113011101F001E0140A0000EE00FF50
:105F50000111011101BF01EE00E001300110010546
:105F60000300000F000F0A050000F800FE030707FA
:105F700001040B060000000001040707FE03F80FF0
:105F800008000000000A000E001F001F000E000A9B
:105F900011090000100010001000FE00FE001000AB
:105FA000100010080400000004800780030D0700A3
:105FB0000010001000100010001000100804000075
:105FC0000000800180010D07000C000FC003F000ED
:105FD0003C000F00030F080000FE00FF010101015B
:105FE000010101FF01FE1008000000000201020192
:105FF000FF01FF0100010001100800008601C70138
:106000006101210131011F010E010F080000820012
:106010008301110111011101FF01EE11090000308E
:106020000038002C002600FF01FF012000200F088F
:10603000000080009F011F0111011101F101E10F1A
:10604000080000FC00FE010B0109010901F901F043
:106050000F08000001000100C101F1013D000F0027
:10606000030F080000EE00FF01110111011101FFF3
:1060700001EE0F0800001E003F0121012101A101D6
:10608000FF007E0804000000008C018C0108040061
:106090000000048C078C03120900002000700050DF
:1060A00000D80088008C0104010401110900004897
:1060B00000480048004800480048004800481109CE
:1060C0000000040104018C018800D8005000700019
:1060D000200D07000002000300B101B9010F000606
:1060E000190D0000F800FC010603FB06FD0505057F
:1060F0000505FD05FF050601FC01F81209000080F9
:1061000001F0017C004F004F007C00F00180010F86
:10611000080000FF01FF01110111011F01FE01E054
:10612000110900007C00FE00830101010101010151
:1061300083018211090000FF01FF0101010101013A
:10614000018301FE007C10080000FF01FF01110126
:1061500011011101110111010F080000FF01FF01E0
:10616000110011001100110001120900007C00FE55
:10617000008301010121012101E301E20112090073
:1061800000FF01FF011000100010001000FF01FFD0
:10619000010A0500000101FF01FF0101010B0600DA
:1061A00001000101010101FF01FF10080000FF01D2
:1061B000FF0138006C00C6008301010110080000D7
:1061C000FF01FF0100010001000100010001160BA9
:1061D0000000FF01FF010F003C00F000F0003C0058
:1061E0000F00FF01FF0112090000FF01FF010F0076
:1061F0001C007000E001FF01FF01130A00007C0099
:10620000FE0083010101010101018301FE007C0FF9
:10621000080000FF01FF012100210021003F001EB6
:10622000140A00007C00FE0083010101010101034A
:106230008307FE047C0412090000FF01FF01210016
:1062400021007100DF008E010001110900008E00A5
:106250009F011101110111011101F301E211090066
:1062600000010001000100FF01FF01010001000128
:10627000110900007F00FF00800100010001800182
:10628000FF007F1109000007001F007800E001E017
:106290000178001F0007190D00000F007F00F001BA
:1062A000E0017C001F001F007C00E001F0017F0086
:1062B0000F120900008301C7016C00380038006C20
:1062C00000C701830111090000010007001E00F84A
:1062D00001F8011E00070001120900008101C1013F
:1062E0006101310119010D010701030100040603D9
:1062F000000000007F010704000007000000070BFA
:10630000064400FF0144004400FF014409058C00DD
:106310009200FF019200620C0686004600200010E9
:1063200000880184010C06EE00110111012E01C04C
:1063300000600105030000000007090500000000DF
:10634000010182007C080400007C00820001010938
:10635000051000540038005400100905100010000A
:106360007C0010001006030000800580030B06105F
:106370000010001000100010001006030000800143
:10638000800109050000C00030000C00030B06FE70
:10639000002101110109010501FE0C0600000401A4
:1063A0000201FF01000100010C06820141012101EF
:1063B000210111010E010B068200010111011101E1
:1063C0001101EE0B063000280024002200FF0120FE
:1063D0000B068F000901090109010901F10B06FCF7
:1063E000001201110111011101E00B060100010071
:1063F000E10111000900070B06EE00110111011166
:10640000011101EE0B060E001101110111019100A5
:106410007E06030000980198010603000098059885
:10642000030A05100028004400820001010B062821
:106430000028002800280028002809050101820002
:106440004400280010090502000100610111000E3E
:106450000B06FE000101190125012901BE0C06FEF3
:10646000011100110011001100FE010B06FF0111C6
:1064700001110111011101EE0B06FE0001010101E4
:1064800001010101820B06FF01010101010101016E
:1064900001FE0C06FF0111011101110111010101A1
:1064A0000B06FF011100110011001100010B06FE87
:1064B000000101010111011101F20C06FF011000A0
:1064C000100010001000FF010A0501010101FF0189
:1064D000010101010B068000000100010001000123
:1064E000FF0C06FF01100028004400820001010C8F
:1064F00006FF01000100010001000100010C06FF80
:10650000010400180018000400FF010C06FF01043C
:1065100000080010002000FF010B06FE0001010131
:106520000101010101FE0B06FF0111001100110024
:1065300011000E0C06FE0001010101410181007EE7
:10654000010C06FF0111003100510091000E010BFA
:10655000068E001101110111011101E2090501006E
:106560000100FF010100010B06FF00000100010016
:10657000010001FF0B061F00600080018001600028
:106580001F0C06FF014000300030004000FF010CEE
:1065900006C3012400180018002400C301090507E0
:1065A000000800F0010800070C06C10121011101DB
:1065B0000901050103010004040200007F0109052F
:1065C0000000070000000000070B064400FF014424
:1065D000004400FF01440B0600008C001201FF0381
:1065E0002201C40D078200450025009200480144A5
:1065F00001820C060000E60019012601C0002001FE
:10660000070400000000010002080400000000FE72
:106610000101020804000000000102FE010B060057
:10662000008800500020005000880B060000200069
:106630002000F80020002006030000000400020BE8
:10664000060000200020002000200020060300009B
:106650000000000109050000800160001800060B21
:10666000060000FE00010101010101FE0804000016
:1066700002000200FF010C0600008201410121011D
:1066800011010E010B060000820001011101110130
:10669000EE0B060000600058004600FF01400B06AC
:1066A00000009F00090109010901F10B060000FE2D
:1066B00000110111011101E20B0600000100C101EE
:1066C00031000D00030B060000EE00110111011155
:1066D00001EE0B0600008E00110111011101FE08F0
:1066E00004000000008C018C010804000000000080
:1066F0000208010A05000020005000880004010B78
:1067000006000050005000500050005009050000E5
:10671000040188005000200B060000020001006107
:106720000111000E0D07780086013201490239027D
:1067300042027C0E07800170004C0043004C007048
:106740000080010B060000FF01110111011101EE93
:106750000B06FE000101010101010101820B06FF90
:106760000101010101010182007C0C060000FF0112
:1067700011011101110101010B060000FF011100BF
:1067800011001100010C06FE00010101011101912F
:1067900000F2010C06FF011000100010001000FFB5
:1067A000010804000000000000FF010704C0000011
:1067B000010001FF0E070000FF0118002400420045
:1067C000810000010C060000FF0100010001000132
:1067D00000010E07FF010C003000C00030000C006B
:1067E000FF010C06FF01060018002000C000FF0199
:1067F0000B06FE000101010101010101FE0B06FF74
:106800000111001100110011000E0C06FE00010123
:10681000010141018101FE020C06FF01110011007E
:1068200011002900C6010B0600008E0011011101A4
:106830001101E20B06000001000100FF010100014F
:106840000B06FF000001000100010001FF0D07031E
:10685000001C006000800160001C00030D071F0089
:10686000600080017C00800160001F0E07830144EE
:1068700000280010002800440083010D07030004D5
:10688000000800F00108000400030E078101410127
:10689000210111010901050103010000060B205A25
:1068A000EC62000003072061615B00000D0C205AC0
:1068B000B66500000D0C205AF15E0000060B205A50
:1068C000275C000000070008000A010018111013DF
:1068D0003831303378717073C8C1C0C38881808308
:1068E00084848782C5C4C7C27574777235343732E1
:1068F000151417120207020802010003010903041C
:1069000002040205030500062024282C383C4044DC
:10691000484C4669726D776172652025735F563306
:10692000320D0A00252D3130732025732573000D9B
:106930000A5479706520273C636F6D6D616E643E0B
:10694000203F2720666F7220706172616D730D0A9F
:106950000025730D0A0D0A00564F59414745522034
:106960003E3E200025630048656C70004E6F20702D
:106970006172616D73004B6579207072657373008D
:106980003C6B6579313E203C6B6579323E202E2E82
:106990002E0044756D70206D656D6F7279004C6FBF
:1069A0006164206D656D6F727900637400436F6E72
:1069B000736F6C652074696D656F7574003C6D69EB
:1069C0006E757465733E00626F6F746C6F616465A1
:1069D0007200496E766F6B6520426F6F746C6F61E9
:1069E000646572005361792074687265652074690A
:1069F0006D6573004765742074696D65007473007C
:106A00005365742074696D65003C595959594D4D51
:106A100044443E203C48484D4D53533E007464006E
:106A20005570646174652074696D65003C6F6666BD
:106A30007365745F696E5F6D696E757465733E0032
:106A40006B6200546F67676C65206B6579626F617C
:106A50007264206F757470757420746F20636F6E2C
:106A6000736F6C6500546F67676C65206469737041
:106A70006C6179206F757470757420746F20636F0A
:106A80006E736F6C65005265616420626174746539
:106A9000727920766F6C7461676500009F59000001
:106AA000000000009D1E0000676900006C69000086
:106AB0006A690000FF000000D9120000766900003A
:106AC00080690000416C000000000000FD10000023
:106AD000926900006C690000CF6B000000000000AC
:106AE0009D1100009E6900006C690000AA69000009
:106AF0000100000089130000AD690000BD690000BD
:106B0000C769000000000000C5130000D269000042
:106B1000E4690000AB6900000000000025100000DF
:106B2000F46900006C690000FD69000002000000CB
:106B300085100000006A0000096A00001D6A00005C
:106B400001000000C5100000206A00002C6A00004F
:106B5000406A0000000000005D130000436A00006E
:106B60006C6900001E6A0000000000003113000084
:106B7000656A00006C690000416A000000000000C6
:106B800011100000866A00006C690000008001504E
:106B90000080025000800350FC3F0150FC3F025037
:106BA000FC3F03502578000D0A413A2000202025A3
:106BB000633A20000D0A533A20000D0A4D3A200096
:106BC0002020473A20253032780D0A006661696C32
:106BD00000253034692D253032692D253032692069
:106BE000253032693A253032693A2530326920251C
:106BF0007300253032783A253032783A25303269C0
:106C00002E253032690025303278203A202569203F
:106C10002569203A2025303278004E4F20525443C7
:106C200000253032783A253032783A2530327800F3
:106C3000253034782D253032782D253032782020BB
:106C400025730000646C0000686C00006C6C000030
:106C5000706C0000746C0000786C00007C6C0000AC
:106C6000576900004D4F4E005455450057454400AC
:106C700054485500465249005341540053554E0064
:106C8000CCC5ED2D1207EE76A609CFA6C6FC205F77
:106C9000FD8D1416A5B8757A3E3979BAAC30388EA8
:106CA0004526943C71EA4D1DFC6918F8374D202D9E
:106CB0005431210C7B81EFB98C658A36C3DF9BAFE1
:106CC0001E308AD6E807680B0BE035688B58BB3658
:106CD0007E32A97A0BFA57FD0296BF98D0985FECE6
:106CE0004861E9BA233F67B933A85C1D8A2E7C202E
:106CF000E734169E180B638521022479A0230040F7
:106D00008133DC942FFB993C5492B0BE5BC9D31CF9
:106D100043B1DDD882327602251407C50DB09AA89A
:106D200040A8A51E3236A06AEE5A06EA4519937BA2
:106D300015D2F935CCA21E7B450630A0AC0C0568F7
:106D40005B16ACD089E8FC6CA5CC73D7F9AC69CEE6
:106D50006D5B587537C847ABC306D05F490DF7D395
:106D6000728C03EE6C76DFD400858D59558EDC0372
:106D7000D6F46B0DECD3879CB706E117A13110EC6C
:106D8000D4887F1F10CA9FC23E76045E1638315ADF
:106D90000F1949812919BDDE16F74461A154A2E5F6
:106DA000ED29ADA66BBA4C0BB86D36E573F54225EF
:106DB0007B305B05AE43AA9562856B34907EA481DF
:106DC000B93B436644837252D0B598FB7C73D9209B
:106DD00076A23A827F51C2274FDC7FBB3A9ACD3FE1
:106DE000BD4DDBE778C921983DCD24CD2698FB0B1E
:106DF0004161E9A65592AE9DC6A681AAC9E86FCAAF
:106E000034249BA239A3319056AC2FFE5593AB5E30
:106E1000AFDBAC7A01AF54C31C2298487CBF2DB6BF
:106E2000D99A44511B39D9D92D9E4153B5DCC90893
:106E30003C66FF4C8B0D2A595B084DCBD85EE3F0C6
:106E40004527E204E16D1CBEF4C273E99F818CF812
:106E500066229A6D0C32D98B088E4F8419611A2FD5
:106E6000C61CFC225919B13550CADEB8B48E39C5DA
:106E70008652776910C45319A4391728409DE89C9D
:106E800034CDE74EFDA3AB571ACDE49B6787A4D65C
:106E9000975534F9F710871B6628B1090B342D96E6
:106EA00097B2EE0A76879DEFC602940373943DD99C
:106EB000D2F69ABD50E96EA6D70ABAFCBC8E6E45D2
:106EC000B0AFC5DDD8214F448AEF678FD6D734C91C
:106ED00020A68C6DC459CD6C6D5171B1691A45A74E
:106EE0009C15BB56A10CF2318E1A0411C7EED93D88
:106EF000CA1EEF4DE5F968A3B5D55CC5C16A188611
:106F000075FA4DE404F0C66E87DBE6CAF97A0E0A1C
:106F1000551644B88DC9F0ED7C1ECD5EF86C7E7AB6
:106F200029CA4820B8C0DC4D72A4F7ACA54A4DED83
:106F300002DE7E4E9E8727BDC8F7A2658A4FE9EC28
:106F4000E338336F6BB7B8AC9AA5FD068DE255B741
:106F5000BD0D51CADBF620490882928C113F4632A2
:106F6000352BBC13E8B2B557CDD73C090B6F55A3F1
:106F7000BA423D2BE47A8C769718A7984009615461
:106F8000979F9313418D0E5A1D57932772739799AC
:106F9000AEC133EF4604FB402A8991186AF0D8C28B
:106FA00000D6DAD984DCCEACB8379BFFA463D0F22C
:106FB000EF862682331593FA87F931DD495CB55D9A
:106FC000AA46C9A7D3C5A3CAC2735E9E8018CD4C7A
:106FD0002D6B9ED6C325B1365C49024F0FF60605D0
:106FE0007FC5E755C164E8195A8C5C4CF4771008EA
:106FF000C2F5DF9CC6FA42BBBF53993A70ECEA195E
:107000007EBD6A59CEC70D345B4A4D88A93DF8F064
:10701000BD47D88FCF48814A793F42D30B3E4CD3EE
:10702000376D49F1DCD59909198CF57D6F5688B912
:107030008AAC2246751DB5B6DD07FC115E295A04DF
:10704000A40861B492D62117D06B6871719BE3A438
:10705000D0A5C4E5F091CEC357A5A372F926EABE28
:107060006A72FF82447D6E09FC643D54AC8B607D86
:107070005107216781A1FDEFEDF97896CA84E72BCE
:10708000A8BD656900AEA6C08BF25EF5D21A1C5E83
:107090006B2D87E1EB4331A0E997E40A55920BC6CB
:1070A00033B8DEE4C2451C86EF3B9B8D38A25BF50E
:1070B000A2EDDE55A4EC8A18EBD67D26EB364049CE
:1070C000A1FAACC50DC5FC8B9D077F22F38D36ADB3
:1070D000E521A2A4BA10559ADE0105298C2340B8F7
:1070E00040BBBF40814AAD7C36E8227E2E5009313C
:1070F00097C1DE4B4BB852B4A196006A8E8BE478F0
:1071000003D5E2DC39170B3E9084B824B2A9F11DF7
:107110003957D43715BD754290AD8BD8BE0995054A
:10712000E7FAE5B1C667D7B191BC1ED46A671C24E3
:10713000219FAD6A689143F3E317B6E4B0630AF6A2
:10714000BE016F16FF8EB9BFB3723A54A98E35FDDA
:10715000033FBB9ECA6FA48BC3F343F5A07EA4DCA0
:10716000FD2761C11C0CE16A7F2CA21A3583B9513D
:107170007A9F471D14855E84E39F79513CE3633910
:107180008D718F616AEA2251E7A255A199F1EA89CE
:1071900086939C2B52DC0E89DCE2862C8749E4B86E
:1071A0008F223F907DE7EF369B12BE3D57610D2544
:1071B0005CD43CEE9E28859E6278FDD97E4C594277
:1071C0004D0267A53A267D30CA309A0D4ED31A304B
:1071D00056C1016FA2ABF1204D17F10CA84E59DB3F
:1071E000CAC16B9706164EC7C61E1E958EEC8987C0
:1071F000092D343A0056B5C6558F2B6456D5933DAC
:107200007586185530533627CCC5E4CD05822759ED
:10721000FF5FC0531407A7DF57CC327CDE66E20362
:10722000718EE0048E78A02F2BDCD8302427DE6806
:1072300022FA86172E26902434CD9ABAF7BE64D748
:10724000E68B3749A3E2905C798382609D4A1F0CEC
:10725000C099460263AE72E10F9472FB1BC1736367
:10726000F6E2D93096439D0E3D180A6727624CC955
:107270005BB0C26308C0AA8F51E44A4DEC6FF3CAF9
:1072800022371E91ADA047E8BDE8EB903DB1B04577
:107290002B4F021C4FFD5C18A8B35EA7BE55D5B995
:1072A0008568EA58E8F308BF02B24E669E96881BCE
:1072B0002C30720FDD13C6A3D83C322FB90C4CA76B
:1072C000B1AD2921B8900C0CF4B68D4D200E15608F
:1072D0007FDC8138D2E58A85AFC1A8EF2D0BAC9257
:1072E000344346E9718546AF20B3EB0E3AC83323E9
:1072F00092D1C0F51F4EEE0C54B6FBDBD4FFF4C3A5
:10730000755A0629156CBBEE593A52F2DB370C7BE5
:10731000B332FFE0EC03A857E58FB6CBBD937750AF
:107320000DEA3EE7FDF697AF4E1394C31B5426E1DA
:10733000914FCEEB43E9997C8E4AC28DD6C2EBCFFA
:10734000F311765AA26BF083EBAAC386858A744D3B
:10735000AC32B1766C981BEECC1B5E7A31A29D816B
:1073600064A0FF211A43C92E56E2155BD51DF426F1
:10737000143E0CB18AE207A477861D0D061177E949
:10738000CB18FC2FE4B58C0B6C676FEB26C2F7664D
:107390002E4F8D828DE5F16CDA760A649234590AAB
:1073A00015B2B8DB330EF5091B373C67927319131E
:1073B00039A1F7A5B694D07C96186B4674BA8BADFC
:1073C00036AB2A98A2FB6F42B1F42D034AECB88782
:1073D00027BF95B92BE53197A16990C25145CB2FB5
:1073E0000FF4313BEB232E0C58CC507E1A13FAB21B
:1073F000514E61D46A417B048FF176BE8F006812D2
:107400008C5FAECE046B19D1DE1068718B65A472EF
:10741000F36D5784586169DF2787A014E6EDEFCD3F
:1074200094AF72A7FB6CD6E86220B90676DFA9DEBE
:107430003071AFBA000E82560F9C9476484DAB9CCB
:10744000B87BF7A5A7758FCC73C5D4E393E02DBBAC
:10745000872A37D4A282768FFF915B5ACEBCF4BEC6
:10746000A5B6107B52FB43B02E8F8EFDF8215A57E4
:107470000C0B7F2BAF5227BD64283C5C05225DE4DA
:10748000F09BFB5760D0D997AE851626ACE382CF30
:10749000F33123B6652463F41EB432756DC326C67A
:1074A000F0FE240DEFDA60108B9FB70B989A9DA821
:1074B0004FE131F45E1BBA37B4E15A8D94A77E6177
:1074C00067AD49D07124513B16F905753076208798
:1074D000EEFAF4DC65C7315F197245027DA5877944
:1074E000DADCFE3C5AB14080EA4132C816CC9799AA
:1074F0002545BFB22F70B3A4683E5BB591B13DADD9
:10750000E7182B34B446AE5CB6ABC5997195BA5C3E
:107510005762198081E27CCEBD8C12622B2AC00A90
:1075200040A61AEE79F06BF69B2F393E17E6438999
:107530004B6233B4DFB0DD983DB0A0F60C5022387A
:10754000708E9FA7251AEE4543E7C36F56BF1548B7
:10755000704B6D9E0591C82269D6183978095EB7BF
:10756000F6AB9C80DDC82E32CC0B9CFB9AD12DB59E
:10757000CF6E9C1DF4AADF9A6E2FD8E6EBF4802A1A
:10758000C1FA7F733E9D3138A0CCD322E7C41621C7
:10759000508976133010BCFA861B2990FBF0EB471C
:1075A00084A67DE096BDF77137C91B9F45F1312454
:1075B00010B105083474342535D17CAE6695698ADE
:1075C000315CEC6981F799E57F93CB24B687B96983
:1075D00080A6987FB8676C8E7CDC9B395C9219889A
:1075E000ABB8EE3621B19240CAFC813958F0F9654A
:1075F0004EDBBCCED225B7B47DC0315051B1C8B539
:10760000BFE321C02E8304176068A78D3636181596
:107610002BC28BB79E3B619FBB8B7506281C6635C2
:10762000C6A37D66B00E3A228B7D57446CDA241ACD
:107630000E569D148F6B18D303FD168601A0905D26
:10764000D043329A7E0833A506265689D49DE5C8D4
:107650002F37B2F132A8858CD6593C710FFDFBF360
:10766000DFBA0F8A316364B4C4CACF1F719BD50FD0
:107670005256E00AD00EE94D748E454345913410C0
:10768000EC348619B58563FFB8755CD67577ADDCCB
:10769000A60C07210767DE6EBEC49368B3275606A3
:1076A000351822CBE4686E4A597BECD0A2D3013561
:1076B00091C72FA309D47B26D5A9898DE5FD5AA9A9
:1076C00048CAD40D23A016A9F90AB56B49F6589FEC
:1076D000CFDA88C44616C0DFF24B159B84BB9019E5
:1076E0008322CA497D6C5030E3A9CCEE2BE77208A7
:1076F0006F2994860C1106351281A54813CE270CEC
:107700002281370B884F4489702E69A8D116703BAF
:107710002D76A8F9D44FBB9E841558F89D363B6E44
:1077200068C9627DC38A75129411A65A77A3776BD4
:107730006C660CF175113F197A6A262BE2744E368D
:10774000E54D3E43E2C0CDF7FD525D7AF32ED97B85
:1077500064A4A4FD04BF5499652DD2683982359F75
:1077600013201E93D05DAB11D69AFDAC0B69F4AC1F
:107770001E5D7E0D82E59D77BED085CC936EDFD7F2
:10778000BE8B367C9F04739EE9875B58A8D88228FD
:1077900061D9C1057612129261F785F5FA1911D5F2
:1077A0003165DB48F9C4A5C8FE76EFE17461220AB1
:1077B00035ABC5E6B13DE74EBB1BC0D330247C3EA4
:1077C0005049ECA51D4387BB97DEB34FD8415ADD26
:1077D000D366D571BB9D062D750BB76C3C0FE7606A
:1077E00003BF3BBEBD3C1782EE4CE24AD9FB66FEAE
:1077F00048862CC9F8BFF84440F867D795517B7A82
:10780000970596C1F7E9C1F5B9F3D6F78A9EBB97FC
:10781000E8B0A611EAD6FDCEC7A9B6960A1E97A96A
:10782000FF5B78D5056B2B575C94DC021A2C3A8FE2
:10783000AD479248B0B7932FFFBB8DF4FE4DE07873
:107840001C02C72C1364BA0AE18F003010E32F57D3
:10785000038D7E9B79A3055C1AE8B600C5EF06E0B0
:10786000A073E444BBB5EE5E1C58954B033EDD426D
:1078700098756796EB2B13C8303B5916CDC9F2604B
:10788000E85E8D0D7C84798804EE306EC923B8C41F
:1078900093D8B4B1AF09611C20CB7FB5B8685E3D09
:1078A000C0EC772042C4D6C5BC8B5F7114405B6AC4
:1078B000B9B3D75B6BC0D021CDD8A55F446EB28E73
:1078C0008AEC76F38B0EDE8B68A8EB608B0B65E79A
:1078D000711EE0B69BCCC274685ED81F628CC85F14
:1078E000FD776FD855DC56FD1F6FBB153AF11DA310
:1078F000F0575318C681E10AB9929EF528D1C7FE08
:10790000E37A155AB14E259723D1C4C07A542ECDAF
:1079100092340C583A70D715C203A4BF504EB60A21
:10792000F1912EA17716FB019EDA7D0089921F3519
:107930005A0DAF6BC9CC2332BF95099E77E799A545
:1079400015FE56041D81FFEDE66E3171944AEEBCC2
:10795000C0E6DEDC5405C33A4EC2A88481DC706503
:10796000779D063CAC7BE08390CB19B30B626CC572
:107970001DDFB814C1C80C25466601479A39CB45AE
:1079800025D15AC9CEB73AE86EDC0AE57B30774399
:10799000F71606F8D3E64F4CBCE02E4681B3D7C5A8
:1079A00018E7CF36C26F85AE788A6854B77F8B3EB2
:1079B0004FC96A7477586F0B6F7E02D050D9871702
:1079C00084C163ED039DB8804512FF762551A44E16
:1079D000D1F32939AE1D9BD960039FDCD0960829CD
:1079E000E08ECB494AF1EEE94323E7322DEBB56C4B
:1079F000243771F7885662E83FACDAF709620879F4
:107A00003F4EFD109F84914FA586F9E5A9E0DDEA80
:107A10004A003FC054E30DCAC8D159978143A9C950
:107A2000674AE467091ECEE9B8D417EE2B36A98061
:107A300038A5A469B5D6B2DC0C3667A8A6FC368793
:107A4000513E8ACE82386C1C4129EE5D047B0A02CD
:107A50000D035AC109C300AF6651921D9858C31354
:107A6000CA20EEDCA82A9067B746B74649854A7B0C
:107A70003EFB601DC88D577CBB881610AA44157646
:107A8000FAC00653A245A3B167CE6EBF36D65E4696
:107A9000CD3EBA3AA92486513D0EF7F9F74767F073
:107AA000ABE5214D21509942AE88A5B365F97061CF
:107AB0008902562222F63BDEAA7B9279B0C85E2F5D
:107AC000500B9D792E0ED8B5307D81FF0267342D85
:107AD000E43EBBCFE344F3FF1BC3339649C43746B0
:107AE000976D687DB5B91DDAF53965CE731BACBFEE
:107AF000704D9BACA9A5A093865353811F07C47BEF
:107B0000C2E5842E810B101B4869C5051BAC6908B2
:107B100090E9F8C0FBA81AF76B623CB508E113794D
:107B2000D055C1FC521FC81C860C7A7632255630BF
:107B3000629C43A33641AE9B8E5F5313970DFC5F4F
:107B4000BB3E7953815D3E5DE8B3B2F1771E14B35D
:107B50005F2E659A29268A7960FFF38E6E14084697
:107B60005354A58847B6ADE801A8ADACE803B2AF61
:107B7000431157AA4848CC90CED0D6D0FEDA9760B1
:107B8000D72BDDDE85E9348386622D717512781E70
:107B900021406F8C35ABA838EE6F78CF9A313E2FED
:107BA0003D6327EBE3F829D1675C52CEC52F9A1BC2
:107BB000B60849A94FB37F7CD4EDE72D7A31C0C414
:107BC000D1BB86C9A6752947F5C55CF6923D4CBD6B
:107BD0004320732429C8B119B12866A559A5B8074F
:107BE000640D92F9DFFC1F0A9285D868B86291A6ED
:107BF000D0838997A1BD1A6BA52890BC86596BAA22
:107C00001EE72B42DDB32F28B5A6AE626DACC98747
:107C1000C9323E3CB3727C6960EB684DFBD21915EA
:107C2000DFD965557FAFBA0E5D073D05C8433D7589
:107C3000DF1FA2139D99BB853D6C73EF59969F671B
:107C40007E7860F9CA8FE5016EC25F49A124A775ED
:107C5000E1F6B184F6BA49AF822C4901A235C8CA0F
:107C6000E7CCA10C5B9BE0FA8576A1AB6599B86681
:107C70004AF14FEA5C01B476D8462732779E19AEB6
:107C80004DFE616FDA939A664BC9CF78AC79F8886C
:107C900029D4FF40890B7296AAEAB4192130FBCA95
:107CA000796C8A89C7EFA8D827DE82CB2EF9635971
:107CB0009665CFC1D86E724A4C39B8D5C983958FB5
:107CC00020936383636B1964A335224C16323554B9
:107CD000BFC8E3498000BC69A10D48B58B0831FDE0
:107CE0002C2AE65896D88E816DE61CAA75EED5E34F
:107CF0001C04B416EC027C607945C321D060A3FF5C
:107D0000576BCD5EA0B13DC228AF46995D6D43D1A2
:107D100024946607BA67D24FCEA599174219AFD7F8
:107D200017222D6BE6D58605DC2966E554BED9639E
:107D3000E10847BCCF8B18A9A14FE0E3981D623939
:107D40000AAF22E802298D181C5A8BA48AF6EE1776
:107D5000A966E1AEAC7EA6AA6A723CC9F76950BEBC
:107D6000F9FA197E63D0D9FEB0F351BC7ED9F1E3A4
:107D7000A8A0E862CD10647377548714FBB4594B04
:107D8000D72813742C7B31C85E0978A56025770D40
:107D9000A2F0DED492D796B963989C76C39037450B
:107DA00075926538702784AE9C8BF7F50902579D54
:107DB00057F0FAA00157365FE542AF8901002E382F
:107DC000F1C8B70D4E5866C23D6DDEB1F4AC068009
:107DD000234B1FDEA8A066B97D87184D8AF5608DFC
:107DE00029A43941076D81399A1F5D780A0FEF1573
:107DF000EA843C7753FF1D0D755737F25C53B0860C
:107E00004F7F3D24AB2F4ED6961011383579F65959
:107E100047A1C0C58B81B09945F3792E85AA5FE74C
:107E2000D7389A3393E199E92CA908B602117B2837
:107E3000861649CBE98A9F5266C27E6FA997AEB17A
:107E4000ADDA70F3BEE2573B8F73FDFA8179695169
:107E500047CEAE782BB25FFF518B24536EA92743D8
:107E60005C1376470784B9B02F1BCEA5885E4D16EC
:107E7000156A753F6EA947D1074DAA7563C41238BC
:107E8000C71F5F00E7F5D2A8928A76D8D691469CA4
:107E9000ED564940DBA3672A5615DFB3547006A19F
:107EA0004FD26548C03959302F74600B2B187CC4F1
:107EB00015DCC5837841B6A4BA26BE871AD986E0F8
:107EC000D43D3E98684FECCB3B2D1366358024EEB5
:107ED00098362FC0BC568DC2DDC6CC96B0CD704B47
:107EE000E6A75D86B04D171C69132CBE8786AAE0F5
:107EF00082629336DD98F7FDEE496CC9818F5EA3EF
:107F00003A5449F2655DCB8629A1CC1CB47799AC73
:107F100099D4431311B2911A4B092F91C007C96B21
:107F2000D4C92E060C522DAF9A9A6D12AF00C654CA
:107F3000B59DB74331FCC35EEF93BB8E46F2272A53
:107F4000D37C111365B345C99282E092FC4009A627
:107F5000C7B2495A962D6AF1C401619C771B92EB16
:107F60008440391A4EF063C41B6C6DE056BBE315B8
:107F7000C3B8C32934784FDDF64E8AAD0131B879E4
:107F800091C2D3A75DEA63D3C60D04895ECC74BEEB
:107F9000129C6FC0EE8758269AC1252B214D9A72EC
:107FA000D14ABF0C1877E358ECFA6FFDB71D32A326
:107FB0004F4128118144038075E538B1D939FDB7A7
:107FC000C72FEFF2187D4EEEC48BEC8D5BAE1FF227
:107FD0003EBA4902A14DE1B4B16A79C329B1F1E2D7
:107FE0004FDC8059A0148AE349713CE52B774EC4DD
:107FF000F844FE4975BD3EBF6D6DEBF8EDAB6BC04F
:108000009524FCB7EA65C607E58F177490163C53B4
:1080100093BD9B0A4F122CBDC415B1D307B30742C1
:10802000D8F4FF9933A5AC851126263CA9442F1618
:10803000A37F778603BD60F002EA89424F7DA4A149
:108040003A5CABCDC110FE37BEC58C90C31F32B3B6
:108050000CFA3FBFFE6241BBE514F1793A38E8689B
:1080600015DDA65EE3C2449DECA67D74AE1E3FA85E
:108070003A0B076F225EBDD397BCA7DF54C5648758
:108080003DC73FFA358759ED9D04A7B00FB3B949F5
:108090005B692DF031D1C80E36BFB606BC02892906
:1080A000B47DFD1F4B81D08E1335C8AB66B2E0277F
:1080B000A6E4656939A211122777A50FB470686527
:1080C0008F28F08EA9C965E59432335DB834168DDA
:1080D000CE438F6070C410F6DBEF8EBE15D4C8930C
:1080E000A6DA077FE5C1A7BA2F736F636C67211605
:1080F0002389AE294291942577CB78B9FFEBD61B23
:10810000A8D2FAB5B157C065E58433F2A4110BA724
:10811000F33569C7AE7FE7144EB40A7D2BFB84A804
:108120009010A664887AB717A0D74CE2940EC6EADE
:1081300046D9B8D780F1340806837512FCB6AA5B1D
:108140007F367DF7A2F8D0311E06D4E8F212D7733D
:10815000FD9DF967FFA3B905CFCA19DCFFD2E0CABC
:10816000C62DE57F8271089102890E895FBFED13EC
:10817000D54EF80AC0C97F5E3A522DB38648907F2B
:1081800004E2A694779FF42BBD1A4F966A86BC38FA
:108190003376EF9BF8660B94A3BFCFC651273DB350
:1081A00007C787D760876BECB19D8BAC0E6FDF483C
:1081B0001EC6A43C0681283C165EC6659D66E3A7E4
:1081C000B0CD58F112FE55354DF4A6A6E8691D450F
:1081D0004D72AB682AA79A7C468A6DF906D296E65C
:1081E000A7A7672BDFB9F6C17083A3C7AED3A7518A
:1081F00004A834E0662AB00155F6CBAA2A374BFB17
:10820000B40403742FD7456105A917369CC58A7A33
:10821000AEEE22C4422F1A8D5B3DA7E2DC75FDF560
:108220000DBE053439EABC634EC85DDCBC0F9CDA78
:1082300031849782DBE83B1AE77EFC88EDBFFEF2D3
:10824000BF294F5ADBDFBCAEF4044D56ABC7A56B5C
:10825000660D43A838EAA0872C34718238CE046BAF
:10826000DB26DEDC161FF28B51693EDA444670C114
:108270003BB4BA7E36AE1A98FB1657D3C2EDDE4039
:10828000FDAA541FFE0000013A8B56B79299646B09
:1082900028D458EE165800812E2AB3BD94857188D3
:1082A000077E03A0026F51E549AC34D6448193E5C3
:1082B0000995C9E3D008E82BA0E663021BD739B4BF
:1082C000227842AD2C41C5EBA21C3715015B048A14
:1082D00097E788871DC78FF921D30BAC24B0446B77
:1082E000310F054E40A90DD9124035570B4C0B4D9F
:1082F0001619672830C5775E42EF75C810A76AD790
:108300009E6EDC2FD95BAA106AB2F706AAF235E29C
:10831000053CE67624AEB102A87449E59D8DA00225
:10832000D09F307ACF844CD2F869A454170AFF2228
:108330002FAFAD792DF91389E8AB4363EB45C93A0B
:1083400090F7CFF35A6A084FCDA7CC0050BC06492E
:108350006263D372CB76E426D308959C94D824B07C
:1083600082913F3C179300F8DA3929C0843D708F21
:10837000C3D12B4FD4BA1FF477E7E8D148FEF49865
:1083800028A68A6AC27E933D308A0E413341277502
:108390000E8DBB2709049E1B25A77CA9EB65491BF5
:1083A000D35B267090612B9CCCBA820AFF1BB65B14
:1083B00089FAB8EB2457B25D80CAB786E61963958F
:1083C000D4868773FDA0B5DDCCF3389E161EC6F0AB
:1083D000800BFBEF0163FF70FB86BD946BD8C5502B
:1083E00024302AAE7D30162945C19D7D1C4BF9C72E
:1083F00084B8C5B972CF0CC20B94D9160BD131C059
:10840000C18020CCE7A69D94F486C626376A3C6BD3
:10841000D253F7729455AE6726BA248A7AA92DD81A
:10842000D084B89392B7EF7373DD44E8F4CB7F70D8
:1084300066C6D6E6ECD30A4C26DF212DBBF2DE68F9
:108440009E8EBCCC6F30983B2A0F4CAD8109F55DF8
:108450008833323357828618445ECBB1FFE54C0334
:10846000CF8BC433D3502ED8568436B4FE7A84765C
:10847000B57C0DCB0F45870E9FF2158AF5C7FF031C
:10848000F143DD2C417157A06139B507E479834B85
:108490002E370339BD17B0F9982D51635DD5D1B191
:1084A0001FED015244C5E3142F156C368622D3D13B
:1084B0003BDEE795F9C78F1F30264B4818BF10A247
:1084C000EF0E5726E9127C5DFE95B7881A5F5BAA0E
:1084D0006DA5C801B68F2C30D8655F487D3AF3DCB6
:1084E0004C2AE91BF22E7F62A7DBAF984CC412D551
:1084F000157D5FA5E8673F6F66353930DD332A5C4F
:108500006C73702EA76333B7D2E83380B64376C658
:108510006231C3E580EB9E77C71285CEDA5E9B5C45
:108520007157565E07DEBDA7DA9B959B5E7C68ACF3
:10853000FD9AAD123AD4818B6834465F9236AF4CC7
:108540000EF35508B5F0FAF47BB87709543CE8EA25
:108550002A62476F8D3DC26A3D4FD11E951B0F8425
:10856000EAA6831140AE3A11B9FDB49F759566EB4A
:1085700004EC22389BDFC4FBE15F1D793B3CAE1964
:10858000F4517AE39323293057AAE937E9D7EB9BD3
:10859000DC45E92DF47786FF1DD71B3B67BEC7FD81
:1085A00051928E46E98064E6B062ED0347B63D190C
:1085B000D95DBC629C0819443BFB558AF838431AC4
:1085C000374FA1646D2A41FAC11D478A5019FC3406
:1085D0008F4869AE1F55EE24BC1C75FEF037F318AA
:1085E000B787E5BCEA72D4367DE60498F56DC91705
:1085F00031F31E86D1F78960783369B0D0F5B028A1
:108600009F60B811447B5742A39CBA515EAE2EC402
:10861000D35FAB5BED4908DC0CBECF4F9CD436B2C8
:108620007AA2660A6DF3A28D7B5E28C9B49C962C53
:1086300088D9D95B2F48561DDC1CD4C3C2E6631E03
:1086400093D330A9121AC6D1BF84EB2B2CC1F98E5B
:10865000ACC3401BF5736685848D690D4A556BD894
:108660000BA1D1A49E6A5D2F0DFA765DE653922987
:10867000751B59F92E99DDB659C23ACF4126A2A3EE
:10868000891A8548957B6EBFF3CE25513B3F3DB39C
:10869000E0A5D3C0A84647B8F3FCD04CCA6F773BDF
:1086A000DA4D7BFBD4FE1904B2AF3660018548B0C9
:1086B00012BCAD8D56E2DF095D839CB859AF0CAD9D
:1086C000BE89FF1C7B3BFE447BEB8CBFEA0209E6C4
:1086D0006C04820EEAD8FC78FDB63352C66A452B8C
:1086E00009F97765F23A6CF24E2A9EC1AB517C3F94
:1086F00062655D7E8F5071E0F70C5AEA93AA988606
:1087000010D084F6C588F2D04F4F5A529A0FE1E04C
:10871000A74ABC173665981D0B03EE2301CFFC3129
:10872000BDF24E0D3A82C6FF67207BF8967E89A186
:1087300027BEDE934BEC5067D66AFDF3C47A100275
:10874000E485DBDA2CB9FFED16D9EAA7CF9DBB7023
:108750000234E13A73198022F3B166C3E09D983682
:108760009DB668C52A4ABACC24E467A1868C9C3C95
:10877000D6FDE6C1CB7CFF0AB9552E8E31D5067EDB
:108780001199E34A512DEC603938DB493FBBD43FA6
:10879000E400DA3E74B807F95C7E111BD334277607
:1087A000A415DCA1B2DF69FA6B992251462EF3B20F
:1087B000C57C7AACC087B6633B13720C59168CFE2D
:1087C000760379EE3D68276471C06A1FFF4E7C8294
:1087D0000D36B68C9E71D566F39BBE43D98FE4BB34
:1087E000D602F9B557CC449C6A640E5483837D0F3E
:1087F00089801F795B46B23F11F5E992DC10A5EC48
:1088000096DC0210C5FE853AC184699D8E8E795929
:108810006912D93B15A89B40DDC7DD358BE2A15716
:10882000343D8E768CFB7A6A95E2E4C193164088DB
:10883000828EA6B5B89EEBD2E39B1C0B9F53B29ED3
:10884000D3DC7EB1650BE6261A32816EA8CE2B3CB6
:10885000947477A4C8E1866D56CC985648EE33A13F
:10886000C76B1F16E0D133D891906E22FB5BBB968D
:108870000D6E29A8C08806BB9207F53DD533B77A9F
:1088800093F774C6911E5CB14896304643955B4B96
:108890007204EA9AE85549EDE016D6A441CD7694E3
:1088A000CC03FC025947749711EDB998016FB420BD
:1088B00057294C8384F5F68BC6D8B6F6835B7402D1
:1088C000659B010BFC6BD38FAAF81787EAF5437001
:1088D000C723E68CEFD0D03F0D8A12AB6108D85D7C
:1088E000DC04616DFC0C927063690D04E160C7C922
:1088F00066DA76405FD0B76AC9720F2839FFE76B36
:1089000032A99384FA758FE3B688A3DC026522DF6F
:108910009CD2CC727EE8831677C8809BE214B97F24
:108920001CD9AC7F152CF185F05CB403B989A52C5A
:10893000393A59530B15C67426370E9A17A3DBB56F
:10894000AB0742962A16A8D731C72760183C377064
:108950000B8CF79FF6CBF35E8F70F74E8F815CBB6D
:10896000973FCB174A1DC133EBE19B7AED4E15695A
:108970001FB6B1943148CC8EAB295112946B03CB06
:108980001AFD61F5C63E5D309088666D3C0957D38F
:1089900034FF93E59273BAED291BF1A48C36DCBD4C
:1089A00086E3025618A68046404DDD7B8B482C821C
:1089B000588B7D683588F9F50944D97127EDDEF1CA
:1089C000CA2E4D2AD706EC9461AAD967061D121249
:1089D000FC8EA5E42AAEB1E021CD950FCF214FF456
:1089E000F98277F32466C1156D207111FC2BE12902
:1089F000CE02389343A301406E6174317869F80662
:108A00006390A774B114E2149B9DDC9ABC3F916AF9
:108A10004C560E66B0EEAE991F7BC132275AEF015D
:108A2000A96F4636B9BB47D27396430B82722CC1ED
:108A3000D83DAF809743A08CB5EDAA3643DD86F8CC
:108A4000C39A0B66911F86E090A52E2D18198C27CE
:108A50000FE6E24F0755F94E238FFEF22ADA110A8C
:108A6000D86680C9B75875973B0E112EB21523B83A
:108A70000E2C700C00A232485BC01531F6059C8BA1
:108A800066405C59121A8ED40DE7AB56865E3822CA
:108A900080444951DB76BA4B3024141B7A78000F9E
:108AA0007CF97F1EB9942ADEDC7DDA4829566F599D
:108AB0007A82274B811775A5D0C1CDA786DCE981C5
:108AC0001B644F4D0A4C21A35042EEBAEE48914D23
:108AD00044F0A8117F79D9ECA5374E02BA8A208ECE
:108AE000E81BDE72AEB5E42B8ABA43952373891472
:108AF000F32BB78158764038375A4E5F274530A15F
:108B00002A8EFF40C5B603A7A98DAAD19C955CAB60
:108B100089DA527C5327D7646843479D611280FFEE
:108B2000E0A8E38CD62863DFBCE8A2EDBEA2439F99
:108B30001AE0945D4BDC1A11AECF2EBDBA8CBE028A
:108B40003EC2BC1F0E3033E8398F3D6CE6B9A71921
:108B50004DC3A6EF985D6555C338784D20A8E6262D
:108B600071B07A0441F565A5FE2525662A1E58DAFE
:108B700065E0E8E38937A3BB7DA41C44185CE706E5
:108B80000E9A62EC507B6F087C3FC9FA7B0EF5A40D
:108B9000BB6563C1BBEE2DAEBEF9188EADA293C509
:108BA000FD9E7415169FA2742B03046B69DFC87DAC
:108BB0005FADB13EEDB4EA5E6C0C15903A037056B1
:108BC000623A475416424A8A2FAD98BF52FA013092
:108BD000952B8295C7F2AF77AB12AB3BF4FD559165
:108BE00081FC272A8FF40174B0B1ABD041D0F1726F
:108BF00089B4E78D2B52B76DA74899345CE5512AAB
:108C00004BD450C77481658160D8F5806AC45C0319
:108C1000D9FDBED6B2F3CA4708A757010494869C73
:108C200076C388D37A4E08CB6672B8C7B43D4E304F
:108C300062E4DE2FFFCEF5412E0BCFD8B64908CF28
:108C4000649233DAF5628AA687A11E06921EC5EBEE
:108C50006B391DC26F353F38BCA6AA18ED87A78BAC
:108C6000348EB8C8D4491B5DD92D4E36E6A8EA52D9
:108C7000E8043884EE9AAD1AD49CBBF40AA00ED551
:108C80006C2F0ED8AF47E1F903FD3C1F67782F5BCF
:108C9000A85276345A73A7276EAB48BD34FDE6ED73
:108CA000545CAF0532800873B24D71DCD9267C8AE2
:108CB000058A6EAFB7FF06ED0C2CB8AE1E92E5CA62
:108CC0005F65941E7FFBFFF9032F993C243AC74C44
:108CD000DBB9BF0DA36040F9FDB120BE3D295BC2E9
:108CE000362837A859376098C0E848F86807B6B002
:108CF0007552D83A7F8744243A64A0CE7E52A9DCCC
:108D0000F5862A22F8FB3E95CE12F6338A57C485A3
:108D1000720A6A51FF73E1955D6C25745999F16B84
:108D2000F00578533ED39B9E172F8098F974DDA2EF
:108D300080693755FE0258223DE8242C98A44465EA
:108D40005B967CADC57CA95D0C043953F9A84462DF
:108D500058486568AD97A0BAE47003EC636CE8D737
:108D6000CF0F0396956408A4923FEC2D4A908E7025
:108D700063E02ACCC61C4A5623412CC8C0DC9B7732
:108D80002037C6A8291B358C866A4F4CEF05F3B9EE
:108D90002103F4DB6BF5B958BC91E62EAE26A8434F
:108DA00067EC0D65B6903E50AFFD8AD99496C077BA
:108DB000E7F847A3E8FC3620B9BCE9E8E7021F98CA
:108DC000AB56623D58FDB1B6C8763B42CE3555E74D
:108DD000F0116EF846713187825C25365D5BFA933F
:108DE0009A8AAA26AAA0622201131CA4C845B2AD81
:108DF0007EE1DB44F1B64A55C395FABEF1B60F6881
:108E00006541604FA5D4DA91FE8BCF043CEBC44D95
:108E1000AA1BA89F705350CBD023C2C111F1664149
:108E2000D2BB95D135D87E2146E46CBFD84DE50C38
:108E30006865ECEB5AB0F4E9435C5BD517E0B3BE70
:108E4000D1BAE5742D669BC787BF4BEEE31E3AF59A
:108E5000F864D82195AFD537A7385B012BDCD998BA
:108E60005F29AA8C376C0AD73F6FF2430B2CCBFCDF
:108E7000BB34DAE1C7CFAC45176836ED44EFDDF41B
:108E8000A9E68645E2200A3E6C3BBA7195BE3FD307
:108E9000BED4F3C4B624D966C2555A9CCEBBD47492
:108EA0000EB1A5ACA9ACE506701033C30541E8FDD1
:108EB000703AC0FA7F6F6036E9D1F41860F4C19857
:108EC000FD81CCFC2AB14C15FA5219C904B648AA46
:108ED000988CE17915882235CA2F4DD19605FBA8CB
:108EE000EBA461D6803ED1A73D44ED49B0AB1F59FC
:108EF0009915B6D75626AEDFBE049A19ACBDCE255D
:108F00009FD3B65A72B1102E80D310971BF675CA34
:108F1000D831D6DCE89CA2F3438A7359915218A445
:108F20009ACBB5B9FC6B19A134C619AABD400A6C1D
:108F300013D39BB66BD5E7D471797D501669062B98
:108F4000E12984286585A6DF9510D3F9CC3429DD85
:108F50003854A62D6A4036CB4ECFA7741BED5DC4A6
:108F60006541FF8AEDC3FCBF4D66C459BAE5E5AF64
:108F7000494E9ECB44616D67ADD991A4B1A3910ACE
:108F8000A86E431DB9613F1BFB5786D116AD8A857C
:108F90000686F83B2DB39742E975E93FC4EAD17BD9
:108FA00076B770506EDAE9B4EAC4DC8ADCD3AA7F03
:108FB000CDBC538712CD28F7D3A89C9C5119D3A0C0
:108FC0001A0D2AA3EEC7F75FD2AAD71C38BAAF246E
:108FD000511B0842E3C970195D25EC70A49EEB1E7D
:108FE0007A412B477AA2AE75E668DEC2E86DBEB163
:108FF00011A41993C49AA679C9F81036CAD4323785
:109000002E26E78A7252396AD8AF9115B01A006AD3
:10901000AE5C229A81BD2D98495445D5B6C7E8EE7D
:109020008A4E243215ED6E7836096109052047D83D
:10903000879E1F2697389D8F3A9D7494A23D79C4D0
:10904000D2550F2C14563515F3D804CDFEC6914CCD
:1090500026A4139E1FE1D39C1DFE392FDE2B0A711F
:109060004527AD989BF0AD38CF63B9969ADF9899B4
:109070007DCB7E5FA459026181248A6329C3CDF32D
:10908000E7CFFE696DBD4BEE4DA134AE6A36D028F8
:109090003904F9E51BF65D9066450D170A360A5945
:1090A00032A1955C171F385997A61E02829ADAC61C
:1090B000F0CE73267085DA588A247E7DD34A7EF2FC
:1090C0000DECD9762405A53F84AE39416A0FE9A796
:1090D00096D4C9291AE2BE65C03AA927912C3E8CC4
:1090E000A57D8544603577DF054FAFA8BEA8EA1E91
:1090F000B3CB28F19352988B9138DDC44359C315F3
:10910000513CA9C34420A9336BB1DBF15499F70159
:10911000E2C9D4224E89D1DC5DCA5ED2843AB4B8A9
:10912000DD7B3BFE94F32A35269A390ED72A0306B7
:10913000659314809D0C53D8DD24F7B7CDAE632121
:1091400050DD8C1FD2FFF28F32F24637314C105B6C
:10915000F980F5A7B3539EAD5AAC68F3BF64251AE6
:1091600053A00376697ACA53ACD263FB7B21F4CE59
:109170005DE886A57C9E78ACF90BAD05BD9745DA18
:10918000999361F5091927CE39F9F4ABA9E1351D99
:10919000864833B298A1EB227843AB165D26911531
:1091A0000DD5B9709187C0AA58D86BC55819601AE7
:1091B0000CAB07B937FD0EC5E185F7D4581B3B73DF
:1091C0004E85D178211F10247192596DA16690B1FE
:1091D00072D021BF9D4BAEA87624A25213F35F4CF0
:1091E0000126DFC80DABD2D4F844611DD363A9E4D6
:1091F000AF0B47B29FFC7683771FFE6D141661ABF1
:10920000CBDDBFA1C6E376DAF5CA556BBA3D427B2A
:109210001261558CB1B74D0B798EE7555CB7D50F00
:1092200052E6B2B51FB4F3AE768317970FD1F1BEF5
:10923000F81B5A3747F31C745059BD95A06671E668
:10924000C75599BE71E3579116E789E6FF91E7513B
:10925000EDEA2EC47377BB30C6EC66AC1EB91E5760
:10926000FD20FA29E4457B9F0912198C66E5C19F10
:10927000C1CA657104ABA2E17B31644C370C14AFF9
:1092800060739042A99934DEA89117C585D09F16C6
:10929000242FE19A21E6C569A2228F486B76370513
:1092A000C949D1A3A1B9B1D070A1DF955030B2970F
:1092B000E0267ED1D155653E915053D369A1D56B3F
:1092C0006C1D5FBCBBB616F3D3980669C026960E1C
:1092D0007D9DC0E7BD73D1664A3BFB6F2A90C5C434
:1092E00088BF0791C546B0AE1269CCE02498CEE3A2
:1092F000FB6EA08127CF3A936D759AE5038C92F6A9
:10930000370F878B8995AE76C1431634B3A5978402
:10931000F027603D11593AD116CD7A3D78F9408752
:109320009EA15EB8B651852685EDC37CD99EF560B9
:1093300040DF9EEF8ECA5161EA5A2E765EDC42779C
:1093400015A044E444546A065C7B2400F8E1E2C9B9
:10935000C38D0073F7F4E761D265E3482E284026F9
:10936000F2D17C41540F0A0CD895B4FBABFC39FB0D
:10937000F0D810AA9377EC389EC73D4191A2C0A2C5
:109380007BF902A5FC487706D62221AF9362AAB9E1
:10939000BF31A2B5B958E322BFBD64A26B8EF59C64
:1093A00010BBD90F2227E2A9497C148D769F3F94E8
:1093B00030F7F7D3F50FDA26B57EB197DC09461101
:1093C000736FB7CD90AFE1A8128682A39931CF4BCE
:1093D000A07718B5D5F0CED825CCB7CE4F6F2DCF0E
:1093E000626A64716269870BDAEE6E070683AB1DF1
:1093F000AE67E9530C342286E98A14EE2355204BDC
:10940000B9EC79A8130947F9150E78EBE4765D33CA
:10941000A240C5EDA22A0E90AC6247610F0ED97A28
:10942000EE21EEDF6671F6515659119D737074543A
:10943000A4FE57707A31C860FAEB4BD9D31414C527
:10944000DFA0514CEFB0A520DFD8F0006863D8430F
:10945000EA0214D134F295FC911B76CD341453B545
:109460005923F624B245B5DA21B9E287A68DFD8CE1
:109470003FF8BCA038886B1386B923AD3277B25859
:10948000ED627E75615CE1E6BF2C0B43DCDCCCD485
:10949000B1C66FE0E4FF4B12611AD011F16F454382
:1094A000152DD3188314DF95809916649D1164EEF1
:1094B000AB10FC1450BB4E89CFAAE5077E5717C5E9
:1094C000C5CFBEC08AC1D5E446295FCC4DB1AF63DC
:1094D000DB488CFAA68C4BE30116109E9B122FD40E
:1094E00071894EB1B2FFB2C103AD9E03F7830A4941
:1094F000C7E49A7EC258EC91415F4250DBCB40E812
:109500001B808B760BEBB17E3DFBE4080EE422FD65
:1095100037BF6AB1419D71BC14C419CEAE42FE275B
:10952000AA21B9EED3973B7291D3E352E746C44ADE
:1095300073AEDCD6689927A992AD59828DE8981E42
:109540009B9345B5B61420BA833D5F28FC02086E94
:10955000DBB219B87368ABB5FC5D4103C5005CC4F0
:10956000B6A3E67F3285CE55E6AEE55296B7444BBC
:1095700001A5AC02A80507B4DC03071F6C73A75F45
:1095800038F2EB92B64AF1C906AD8EE9E0178E22A9
:10959000C7A78B698C6C9989D8674D35B2852FEA3E
:1095A0004CABE73EE48351DA5283CEE2AE205B70EF
:1095B000E6A8FD08F18B1E39666B738E75C1A5B8E0
:1095C00005A3C812C8CFD47231C09A122FB0FEF1D1
:1095D0008B05CC00E918B98735D15E060B57D21838
:1095E0002C1A30E5FB83D644A8ACFDAF91AE8F8E2C
:1095F000FA1A161B768FA340B22F981ECA8B885773
:10960000C7AB8CB8587148C895880BDAF62CC26382
:10961000E333769D9DF00F20647415BEEEDF601776
:109620001F6AA35AF7AECC60DDA4835F68BA18380E
:10963000AC27BA96BC28785A99FF89BF3529724958
:109640008D9CC4FC41874C4E66C0F21DEBFCDD9541
:10965000822D3A0EDB421FFA74CA9CE39D36AABAE9
:1096600066F4390703839F1239C252E1EA41546C10
:1096700077669686FECF22A0A57ABAAD22402D0F3E
:109680009CA60701A9B6A19A8B523EA0DD9A30058F
:10969000DF991CB9DA7E26CEB9E4A1B8BF90F200FA
:1096A0001ACFBC037532CEE167052C6527D0E103E4
:1096B00074023CE7DBA4A7D8DEA708C56801A53E75
:1096C0005347982BB0A6694784D694FB418EA707D1
:1096D0003A0E5A6AFDCD14F6C1E2141B2815E71D97
:1096E000A10E5CCDD9D4E8AC6C5C431409A159CF70
:1096F00061177FD45F818AAF1B45C4F5EFA51CCDF0
:10970000E1A1AB59B742A01F7B692328636BFBA87B
:10971000F5A05A5E397EAA8B97364DD2B6BDE0DBF6
:10972000AA49921FFAB0D238DAF116F32A84550BFF
:1097300007F341F91B8D3C4CDD845E377A7E57760A
:10974000F8002A8A19CA7B2F6A319C0FE2CC9A95BD
:1097500051F13E4F54FB03E7F5F1C9A7AF41229306
:10976000954E2F99E02E2D13F03526459014A532F5
:109770006C10A2346E2ADE85D859DD9D2B4CD8EFB3
:1097800021DE68652E77B21C564C50BF6788B783C0
:10979000462ABD1D42BB21A16F918E4411E648B1FE
:1097A00047CBDB360FB9F0C3A6F9B0A4FC2FFCE021
:1097B00018472B35AF8BFC8F8C4102CF55F25DBE25
:1097C0001659D844F9158E4D570947A1D28D2DD57C
:1097D000ACF9C89C9183B6FAB95F5A3EEE4D780158
:1097E000027E7880C0DB092CFE4C1B677350B6BA32
:1097F0005C0F71E04D36FA026B1293D0E1A7393954
:10980000DAB4A050C1CA160BCEFD308B3714DB0B77
:10981000618D6377669EF58F7D9B75B2A080FB8F0F
:10982000374358259DF477D0B3B775438E121E1970
:10983000D297D2F065E304D5FB604DADE5443386A5
:109840005F66FC40DA19B655DA948F0FC06336FABA
:109850007E087B2E0D55912EAA0775F4B5F3D24ADA
:1098600008E9A41F1C2F29D2E50EC5F0662596AC89
:109870002E13F2748104E986B65269068584E5FBED
:10988000C73B54021EF957273121F8D867B6189EF6
:10989000C43AA1F848C23DE6F0AC946BC90FE31F8F
:1098A000A30F8626B8DEC85A64724E281E4821B41B
:1098B0004CC77809EBA5F80281B17C94D6B15CC1A4
:1098C0003C4934FF98F3F84BDC0146B66398AFD0BF
:1098D0002AB629E8D0633590026E5BADB0E2DE7542
:1098E00036FB6C7F94B601A7DF06E9EC4D2AC9D19F
:1098F00066D4DEDE6A98351D1C771241ECED67AD4B
:10990000C53B6BC025DD25D8B53D154848A57D6014
:1099100098C01FF3D3A06074FF4BC79943F9A1FB14
:10992000E14DCAB3DBBE196E5300E1C0C5D4DADE27
:10993000C2F8DA959E09588FB3FC322410E2DD9B01
:109940002560602F62E4737B0083E7298983A0C3CD
:10995000C9D8EAE0959F81CB78A23F4FE1C1840747
:10996000ADFE03C3FBAB3A4DB13E8422F0726032D0
:109970005A3D536772D921AF745616ADDB38FFAA32
:109980005D1CFB9DF21D84A36C5E24F56323F43EF5
:10999000BBFA61E50038ED8A2998F426EF3233E00E
:1099A000148698972E9BE87EFB017E431A5B40212C
:1099B000EC5878A142729A2EBF412D9827617B13F3
:1099C0005BC85BEADCF450BDBEE3D585011EB7D8A9
:1099D000A1FB5F201C27C18BC4B72E78636862FE91
:1099E0008FD2F353E2532769D56BEC4E6F7CD52FA2
:1099F000277F844D4727CDB333777E6EA4A6E7A596
:109A0000E4DB0F53970CDB1747F5E567B29FEAAC31
:109A100031A04B024B0141CEBA4A4B58009DF89100
:109A200011AC527820068A29F62CA18864FCA8374C
:109A3000481EBCEAEAA8F640A799393564DB9C24A5
:109A40000248E94C6F40CB1EEB979F381983FBBA55
:109A5000A80AAC1E45A14EDB1021651F78A716B6DB
:109A6000D521443A51D46BB88552A17A61FFD439DB
:109A7000C883AEFB9AE6CFC7E45A68D43C64437609
:109A80005509BCB350168FB6325C65093F4D925BE9
:109A9000534F9439FE4AA4AAD1447C022DC0B7BCCE
:109AA000D9292365C54821D39F5810F49AC3ECF5F2
:109AB0007E6CA1800EAF7F24541CAB2F64EFA13EBF
:109AC0000D08CE5628C20AF97539298B4E52AE8937
:109AD0006BE74A28D1CD52FFDC8957904AB89F1EC8
:109AE000CC3875D9BEEA3DE54315A6D11E13E79FD4
:109AF000DC39A9BFB7FC3AEFEACD998DEF72E5D515
:109B000083768AB2CDC7FE0719124ECCC83A952D7E
:109B1000EA5AFBAD98BE96BD22ED5E72563AE2243B
:109B20005E2F8905A52160484C22BB89E0B49F8245
:109B300002A956B1DD081D44466D6E5F48C6ACA94A
:109B40008ADD3FC126D57C6AA327F80D4A335D47DD
:109B50006D2058303AC5C0CDE0B8A1E1B74BA49C08
:109B6000AF07E6E757C7047090718E935D779285D3
:109B700027293852E9A9FD8C9EE7AA8AC77FEFF111
:109B80006653F634BE0B26386B2CFB39153BCB9550
:109B900065B283F9C25B03670CE7FAE559FC2E2F27
:109BA000543EA6E4E26EEA33A5B5DCB3B53207ACA9
:109BB0000A1D7618D131D71BA4AB557C4F0F361137
:109BC00069D1DE066AB7FF392F04E1D762F0026A75
:109BD000125362BB46348E287B5CDF744641B17BF6
:109BE00031FFE62F9809712C47372CFF7390ABDBC0
:109BF000A85F68D7FEECF66018FF11E190D999B91B
:109C0000CAB62040750E4AFEC72B8D5F0186E4F56B
:109C10005A266B012619E26797ECBA98EF0905C935
:109C20001FFE179D9C827C117CB844C8080AB64769
:109C30003B77B691290A4ACDEBF8E3A91A7C4AB7DB
:109C40009663C84920F65997268C376166EEFDED7C
:109C50004A409870F8B1D7DF08AA3D683FECFC8A0B
:109C6000314967E3AF796A7FD86987F6382D4E3975
:109C7000E6DB7D96A2F897414D734A240AB47B50E7
:109C8000074A420778AE4029FEFDC091C33D777A6E
:109C9000C3690D7C7C2A39F0138A2B78DD7E541A37
:109CA0000766A5A2CD6F030F883653883A16F602D1
:109CB000DC8B2E8B7D8F03A08756351C9FA91FF947
:109CC000AFA240F7B0948849D913134F6F6F24990E
:109CD000F297C394CCD15D274FD06CB42C4FBDE626
:109CE00025DC69C41079F09A59B2843A38946064DA
:109CF0005ACC4B818AE5E88042DCC56A66122805A9
:109D00005AA52AC72B810B8D1637AFBE6AC43ABA43
:109D1000A889E5DEDD2082F99E860A3600DFE98823
:109D200081D86AEA11BB50844AB61D2045C8EF812C
:109D3000026D66C7BB27E2F6C16F7D4E181AB21ED0
:109D400087E2E9243B5ECD847ACB67CA6D62C2525A
:109D50001AB065734B363CBE5D417F984087BB7D32
:109D60001B4BD1B53AEB3DA07D1420405239DAFCB3
:109D70001548FC3D521250938F91A886A9BC182F0C
:109D800010A1601C1C4FD93347BC066C240D486FD2
:109D9000D30B87B55D9BC2C06617831017767953C6
:109DA00050CB20DFB1441F292E3014E0FDB41464E1
:109DB0009AFDE23541A2FF362D0B70197CFABA17D5
:109DC0005E377A73EF3F9732D0321DEBC78C70ED60
:109DD0004E36193D0F38A40FA46FA296D24983E5E1
:109DE000B8B241A29BD00B5D2299242523D4A43480
:109DF000E43328AB3AA4EDD15596082CEB4D8140C5
:109E000047FB9066A53993E47B309A056567DA597C
:109E10003B997256497B75F4EB1681F486DC7ED053
:109E20002ACC4A24F5F380023E8CBEF1B92B325E77
:109E3000DD02B0EB4EB65503EC5C841121F2262A0C
:109E400004DDD86A7D00E206FD73FAA11D5AD8ED43
:109E50005130562DE34953C1865957021305F6F484
:109E600041BE3A30E90C85398A1D983805048EF3D5
:109E7000642C196CCA66387288E78E75EABB7C9BC5
:109E8000166D86513C7E53BB5A25FF39E353A0889B
:109E90006FAAE6DDD288AD79717B1A406C76C4D3A7
:109EA000940A0481F3F7F8E973DA937E2E34DB1F0A
:109EB00071183E417E602420A8E54B2678CD53AE34
:109EC0002DF31E019A594EE04AFE93A259C67EC850
:109ED000C76CB0B83454907406ECD82A18AAA615EA
:109EE000CB568274B4052F418F6AB6F3974A79E155
:109EF0000585319EEACD50D006516F8C45AA056884
:109F000060AE77CEED655C6C264217920AA4BC3732
:109F100072E96D4C0F34B78209273C72AA85E1A320
:109F2000B7A6219194BD9930C5CC7D443D6E33D008
:109F300092059B2233502DED55066AE4E7032A1063
:109F40009ECCAFF116051E21B47C8773EA89AECC96
:109F500088368832F31FED2DD5B76933109C9B707E
:109F6000102EF446447D6438628B18D59C6F3FE216
:109F700069B5B923DCD74B3182FEBB9AB4DE4A49BE
:109F80005EE9564EC658795178AFE1C68E8A2F7B6E
:109F9000383E7B744BA3019C2E172C0DF19D1E4364
:109FA0008665FBBD8F251F11A3383D42A4195E14A1
:109FB0001802BA3F14B1DF35F68594D03071375AA4
:109FC000BECED433D15BEB9ED6C8260B827073C94C
:109FD0005786C2590C6B1606F54BB567F452F69EC0
:109FE0009FBC46B1308CC1ACD9E4A32332D29A32A3
:109FF000FF311AB247F98F6864FB3FF105BD0C933E
:10A000009E6C79AB72FEC8236BB0A72D517DB78FC4
:10A010005C1004819CE895A737FB4E2D4FB6B91C08
:10A02000DD21663570FCF2371D78AF9DDFE73CBF60
:10A03000A0239DCDF796457298BF9937B710819CA4
:10A04000E0F2C36EABBE03ABB7D12218FADEA27743
:10A050005B3AFB55A0F6831FFC89AA89939B5D6A36
:10A060009F2160F4B5F4B0694DF686405F4A3E7DAD
:10A0700002E4129E7D36488871752D377F7B37CC80
:10A080006E021737B85A59C37E0004E8D6FB0D7F1D
:10A090009C3CDFCB6B1B7818FE2122B00067141E9E
:10A0A000E4DB6D0B99173683EA42AE9B555C1A5779
:10A0B0004550871D20578EB3FB384E80255E2DAC52
:10A0C000969CF078BF7E57423126EEBF202AA387A8
:10A0D00002E49A1C3231B6BCC6922A13151AB27C1D
:10A0E00082A7D25BBAFC2E6D98A4EB9C45B14A7056
:10A0F000FBBFF334B8F2BA0AFDC334B41C459F4029
:10A100007B95F6B111A81A0EBF3F012D857B21A9C1
:10A11000C7F25E3B896C1A447E11602816CDBA7373
:10A120009C40B1596BAC2C96C3EC20FF99D65AAE2B
:10A1300085EE4BF7C51EF5B6C3144A0FA76D44A6AE
:10A1400044FF574B0D132FE9FE7ABD8F9019165916
:10A150003E649CE989942F09F6760415C7864892D7
:10A1600048696147D6AFD671B849ED6B754AF82A90
:10A170005A4F69375CEC5C64F13F1DAB9802DE1905
:10A180007C97DB53E131D9D79CD3A799CF335712B2
:10A190001D951B911F0653FDDCB01D38CA121ECF42
:10A1A000C2833975416D1C6A25B3AA35B334623652
:10A1B000371557F29EC1E089D15BBA46BD3B923F4D
:10A1C000DB2CD0A2DBF83AC2AE0E10AC8D87CA2FC2
:10A1D0005EE6402CC27AB699CE14F0884F2D966870
:10A1E000F976D5073E3B5AC932C840CEEE65A41574
:10A1F000316AE92211F1F117BF8021DA9D2CA2E822
:10A20000E26F7E3A8ED8F2C3F54B34788A75F28AC3
:10A21000BB8DA9E0F9C718A80AF8406394AF4810AD
:10A22000F1808D9CB121785420C5EB35CB3BC89A89
:10A230001C5F8E2A2B122C1FB249603A6C2A834C69
:10A24000A355F53A644076E456ADF198C265D9AEAF
:10A2500013AE2E30D5476BFFEA1CA842EE20609C5F
:10A26000FFEEE2D7B04A1C7C8E691F64C9E5C56663
:10A27000FDB9DF53F931F2FFB707C15980993B1C93
:10A280004C01307D101FDC72DDB8D2D6D41B4F5C80
:10A29000E17B84959B910BF6D11F9FBD9485FF03B5
:10A2A000D4CA9B9014867F314D9197B217560802FD
:10A2B000F84197E841A933F99A2B2BED1E3AB3B92F
:10A2C000FB819F8137C519EC9946F5D96D8EE85E03
:10A2D0009DA9E4125751E887A12B07CE518C16098E
:10A2E00032E7C291FEA66E44A79EA3C4470ABB50A4
:10A2F0001216CE7B446E2FDBD87A4D8CEDFF302EBC
:10A300007A8E701EDDF300D13460E2818AE26B3A0E
:10A310006862FCA52832E2F7285EADC29DA2ED1F5F
:10A320000711C38AED7F50AB4AC998FB6DF4E70370
:10A33000D840904E4D04A180B6733FB2EA53AE8C24
:10A340001D33A72F70135DA52232DFFCF4F56CEAF4
:10A35000794C76A1EC25030F7C6E7134DFA578BFB4
:10A360007F50958D6C395CC448158DB95800709537
:10A37000F7CE2C385D37F2E9670CB8D31D3B2D8240
:10A380004FEE42436FDFE389C5281D3B3896233BE0
:10A39000CC3362A2AF86D35537CEC84093FB1F297A
:10A3A0000CF8F4E7F0EF38766FE53B2CB7BA47745A
:10A3B0006D1CBC08CAE24622A85FD85AEA0A9F541C
:10A3C00054DBA8EF882F2D55FE3723CC5AE5F071CA
:10A3D000EAFC6C939095F6D8AB36CEAE6DEB07B237
:10A3E0001B559E0808AE0E71F2B57419B0EE87D3F6
:10A3F000625B7743624EBDE65D316C07ACDB225396
:10A40000B3C2F0FE68C612DE1EDE2C32792632DAC6
:10A4100061A9B9AF3F6374AE233E64AE0A8CE28C8F
:10A42000BA055C39AE1F8AD4A2B361CA664C24DE79
:10A43000BEB50A0503F85E3F67232CC83DE4D06A29
:10A44000C314E408EB56CF3907BBAA4DA2B288FB70
:10A450003FAE7D1D3931E5EAA416A5F970609CBABE
:10A46000E7646C956DD4C1CB00C81AF5C2EC6527C2
:10A47000AF7145BA1D62C9AEA212D0D4B3BC840A72
:10A48000A37DB78F664853586DF58CFAD2CFC6FDC1
:10A490005A5011062048B6145604AE51F4F6B8814D
:10A4A0004D15706716AD0BC3EE9753CB0ADF8325AE
:10A4B000B18EAA42A94DD7BEF24FC35C3652A795C2
:10A4C000CDF87A07110A352A03E4B1559F44F80FF5
:10A4D0004F75E13A840B11E0D8CF058623A0745F55
:10A4E00056AEC5D13766A484FADBBAE8C6E1B00A35
:10A4F000E50A7FE6A227C6FAEAB630E15740FFC276
:10A500005F92B35C8654D2D42689E4BB9ED0BE1F32
:10A5100006B467F9B51BA7953CC142C56605307006
:10A5200086D2E7D2C238F0775A617116E03E173012
:10A53000A22923F2318415A4412EE78123ABA4A2E2
:10A54000F6FDE466F5686D7CE078606B300068DAF3
:10A550007DD7E00F1DDA7A6D4A378811A7DA1962C4
:10A56000C8084418DB14D3DAC954F684D6D9AC81B0
:10A57000CED83891FC98772D28AC41D10C2A36FBE7
:10A58000841591486E387EE764E14E51687CF2692B
:10A59000865BFF1F7141D7757346FA5008326ACC4B
:10A5A000E41C03CA4D1938A3476DF3184103360A5A
:10A5B000F6BAC1E06E29AF85F03AEBCD222DB3D7C4
:10A5C000C9E6C2E4DD438AB0FBF3A64BAAA5949684
:10A5D000C416426A5828F72E4CEA0325495AD3A4D8
:10A5E0005042528EF4168E3C8F0670A4E0C4A473C1
:10A5F0004A88BE0BFB24838BFA62533A1F18BF1B99
:10A6000009E5C14400CBB3BA0E63CB7925DAF12E4C
:10A61000D9E701B5DF3623892DD63ABB3FC2691D84
:10A62000B2434560EB2EBF24FEF546856830547D6D
:10A63000A9C74909F1741CA628BA6C897CFFDCDD26
:10A6400082CFBBF32F3C0B2A225FE1A6C791CD142A
:10A650009B530B5C79CDB1996896E2DC0950F5A467
:10A66000DCAB2287B1FFA39C04C7748319D2A30A71
:10A670004C58ECD197587B84590A0554C8B1C5C2CF
:10A68000DA52AFCE3C1D5FCE2AADF3B3016B2E93F1
:10A690007B3FE77A9BB8EFDBD41A981C1A477E29D8
:10A6A000BC25C3B9FEE196EDC4A8639661B4DDF59F
:10A6B00052B868887E5A91BB8BBF7DC58F77849CCA
:10A6C000EB1A36FAF34D4979D5A3904DFA878505F3
:10A6D0009E283676B09DD5EC05B7E9C9E4FBA8BD48
:10A6E000A0291BA15E0D63D4D1DF3F474CE512CBFF
:10A6F000F72FCDF7B9D7255BE41990C0CD82EB4099
:10A70000F914ADAD5C9A6D632BD1724201E5152A47
:10A710007C66D9851C2458D8431D7A76F7D129B890
:10A720001FB1F4324AFF0763ACB489A08730A63169
:10A730002CACD29CEAB9BAB4CA73A23378F46FCD08
:10A74000F5195A973D762DF7BE79F01B80A7EBA03F
:10A75000DEFC94BC5295DCDFFC9275D9FBE60FE180
:10A76000189070F2845B729E63761898B656E1C3B7
:10A7700044DA5C9541B0367BDA57F016459ABB1F38
:10A78000877DEF940659C637FD2694038211F4E1C4
:10A790001E0D272249AA1367C8DEFC88A99F5DA663
:10A7A0004B3E1249C794DCCFD6492A73503DCFBEE9
:10A7B000494782C3528F7B28F3764D0A68AF105801
:10A7C000D8B63360E3B7B187D82E9D161998AA0F73
:10A7D000FCB10B6D0A78F414D2C445C4169ADE6F2E
:10A7E0009E6300326839BCCEE62605880D6B79F28F
:10A7F00044038D201175C5E84AEADC92DAAE0ABD41
:10A800003A5AA11B832C56FEAA63D33C69EEBEDBE9
:10A81000217453C66A98AE262F78618DAE3B861B95
:10A82000D268F2BD31A6642F6773B60595E73A7614
:10A830006197B879E1C728CF617A74382BDF5C580B
:10A840005AB94AAB13F9386A958BA213E6B178A9C5
:10A85000E6098190227CB2AE47CFC94DC1A33293A5
:10A86000983B2FA71C6E1066C989804B4D2CC49E47
:10A87000C1B9C548853CFE4820D05227FD4A66AA8A
:10A880000304050A08060BFF0209070D010C00FF6F
:10A890002025692025692025692D2569002020258E
:10A8A000633A256900202020205F5F7C004D454DE4
:10A8B0004F525920434C454152002C0061004469DD
:10A8C0007370206F66660D0A0055534552004600AE
:10A8D000424547494E0052414400442E4D590050D4
:10A8E00052474D005553455220202000662020003D
:10A8F00067202000424547494E202020202000525A
:10A90000414420202000442E4D5920202000432087
:10A91000202000081C242C4448586C7403000000BC
:10A920000100000005000000FFFFFFFF4D000000D8
:10A93000FFFFFFFF0F000000F4010000040103010E
:10A940000201010411040F0417041601180100008C
:10A95000E4A80000ECA80000F0A80000F4A80000A3
:10A96000D6590000FFA8000006A900000EA90000AB
:10A97000DFA800000502050804080B08040405010F
:10A980000504090809040608070206020402060174
:10A9900006040701030803040C080D020C0203025D
:10A9A0000C010C040D010D080D040802080807082D
:10A9B0000202070408010804090209010A080B023F
:10A9C0000A0201080A010A040B0102080204100825
:10A9D00011021002110810011004110112021201DB
:10A9E0001302130812080F081204130113041402AF
:10A9F000140115021508140817081404150115048C
:10AA00001702170119081A0219021602190119046E
:10AA10001A01160816041B021B081A0818021A0449
:10AA20001B011B04180818040B04202020202020E0
:10AA3000202020200000000003000000C9A8000022
:10AA4000CEA80000D6590000D0A80000D6590000BA
:10AA5000D6A80000DAA800001F6C0000DFA80000E4
:00000001FF
